:046EC3000100013099
:10694E00AF50055074D02FF582E4341DF583E599D0
:10695E00F022D3E5309400E52F94002290000FE052
:03696E006403229D
:0300030002568022
:0B568000C0E0C083C082C0D075D0081D
:10568B00852E82852D83E493FF201304C4540FFFD2
:10569B00430FF08F80C284D28500C2870000D2876F
:1056AB00007580FF7580FEC284C28500C287000032
:1056BB00D287007580FF30130CC213052EE52E70B8
:0956CB0006052D8002D213D2A8BD
:0956D400D0D0D082D083D0E032A6
:03000B000219EDEA
:1019ED00C0E0C0F0C083C082C0D075D008758CD85F
:1019FD00758A92D28C124182126292E531D3940093
:101A0D0040171531E53164056009E531640F600358
:101A1D00021BFF126B73021BFF753114E54ED3943D
:101A2D00004002154EE54FD394004002154FE53AA4
:101A3D00D394004002153AE54BD394004002154B68
:101A4D00154CE54C123B821BF1001BC6011B9E027F
:101A5D001B76031AF3041ADA051AC1061AA8071A17
:101A6D008F081A760900001BFCD3E52C9400E52B9A
:101A7D0094005003021BFFE52C152C704D152B0205
:101A8D001BFFD3E5379400E53694005003021BFF8E
:101A9D00E537153770021536021BFFD3E548940064
:101AAD00E54794005003021BFFE5481548700215E9
:101ABD0047021BFFD3E54A9400E549940050030209
:101ACD001BFFE54A154A70021549021BFFD3E52A93
:101ADD009400E52994005003021BFFE52A152A7096
:101AED00021529021BFF7885E6FF7003021BFFEF2D
:101AFD00B40105900524801BEFB4021012696040FB
:101B0D002FE53015307002152F021BFFEFB4030CBB
:101B1D00900526E0F52FA3E0F5308028EFB40412F0
:101B2D00126960400BE53015307002152F021BFF56
:101B3D008012EF64057003021BFFEFB4060C752FC6
:101B4D0002753058788506021BFFEF6407600302AB
:101B5D001BFF126960400BE53015307002152F0226
:101B6D001BFF78857600021BFFD3E5399400E5381D
:101B7D0094004008E539153970021538D3E53C94C9
:101B8D0000E53B9400406BE53C153C7002153B8035
:101B9D0061D3E5579400E55694004008E557155775
:101BAD0070021556D3E5559400E55494004043E575
:101BBD00551555700215548039D3E5359400E5342B
:101BCD0094004008E535153570021534301423D3D3
:101BDD00E5339400E53294004018E5331533701267
:101BED001532800EE551D3940040041551800075D7
:0D1BFD004C0AD0D0D082D083D0F0D0E0329E
:030013000245C6DD
:0D45C600C0E0C0F0C083C082C0D075D0102E
:1045D300E545C39450400302466620230302466622
:1045E300300C03024666E5A0540FF5587D077F01A2
:1045F300124E3A5046202243E545700CE558B40C60
:1046030007201004D210805B20032A2010277F0F7D
:10461300126E5390000FE0FF64016004EFB40304D3
:104623007F80800990000FE0B402057FA01200167E
:10463300754202D20390053CE0F53A90002BE0B5B9
:10464300580D7D087F05124E3A5004D2258014057B
:104653003EE53EAE3D7002053D14F5828E83E5587E
:03466300F005451A
:0B466600D0D0D082D083D0F0D0E03262
:030023000263A1D4
:1063A100C0E0C083C082C0D075D018309819C2989F
:1063B100E599B40A0812694E755000800AE550C388
:1063C1009490500312694E309902C299D0D0D08274
:0563D100D083D0E03292
:03003B0002491463
:0D491400C0E0C0F0C083C082C0D075D018D4
:10492100C2CEE546C39410507C302479200C76AF7A
:10493100A07804EF08800123D8FDF55953590F7D64
:10494100077F02124E3A5035302232E546700CE5AF
:1049510059B40C07201204D212804A2004192012E3
:104961001690000FE0B4020F7F0A126E537F80127F
:104971000016754202D20490053CE0F53A90002BF6
:10498100E0B5590D7D087F05124E3A5004D22780BB
:10499100140540E540AE3F7002053F14F5828E8359
:0549A100E559F0054698
:0B49A600D0D0D082D083D0F0D0E0321F
:104B7300E4F55AF55B755C1E755DFF855B82855AAE
:104B830083E0F55E635EFFE55EF0E0655E60031261
:104B93006EC7635EFF855B82855A83E55EF0E065E1
:104BA3005E6003126EC7055BE55B7002055AE55D47
:104BB300155D7002155CD3E55D9400E55C940050CF
:104BC300BA75985A758921758845758DE7758780FB
:104BD300758CD8758AEF75C90275C808753D1E7541
:104BE3003E60753F1E7540B075B701D2A9D2E8D2B9
:0F4BF300AA75C64C75EEFF75FEFFD2AF12669F16
:014C0200228F
:026EC70080FE4B
:10692B00202F0F90053AE0F54EE54ED39400401220
:10693B0080F7302F0D90053AE0F54FE54FD39400DB
:03694B0050F922DE
:1068E30030300AD214900024E04420800DC2147F7B
:1068F30008126E87900024E054DFF0FD7F247E00B1
:0469030012636B228E
:102F1A008F70E57064017029202F047F018056208C
:102F2A002F03023015123026400302301512302EBC
:102F3A00500C12301630140302301502300B022FD7
:102F4A00CBE57064027020202F047F028027202F97
:102F5A0003023015123036400302301512696A70C6
:102F6A0003023015022FE5E5706403600302301591
:102F7A00202F057F03026E87302F24123026501F20
:102F8A00123036501A12696A601512302E500B7FB1
:102F9A000A12303E20147402300B7F0302301230C2
:102FAA002F2312304C501E7D017F02124E3A4015DB
:102FBA007D017F07124E3A500812301620144C80B9
:102FCA00407F018043302F1712304C40127D017F21
:102FDA0002124E3A500912696A60047F028029304F
:102FEA002F297D017F01124E3A502012696A701B07
:102FFA007D017F07124E3A500D7F0912303E201490
:10300A000AD2300268E37F01126E9A227F09126E99
:10301A009A900536E0F532A3E0F533227D017F016F
:10302A00124E3A227D017F07124E3A227D017F021B
:10303A00124E3A22126E9A900536E0F532A3E0F566
:0A304A0033227D017F01124E3A226D
:104C0300C2957FFF126E87124B737F071262C950E2
:104C13000512003E800312604FD28C7F081262C9D6
:104C2300500512424280FEC22A1268049000D1E06D
:104C3300FF7C117D00125BCA125D3D90000FE0B452
:104C430001051228A2801090000FE0FF64026004A7
:104C5300EFB403031232AF123C89301D11E54270E9
:104C63000DE52754A060077FA0126E53C21D7D0778
:104C73007F05124E3A4002C200E552C3940A50BB6C
:104C83003014B8E533453270B2C2301268E380ABFA
:104A4A00EF253EFFEE353DCF2401FDE43FFC22AFCA
:104A5A005A7E00EF2403FDEE33FC22E53E255AF58B
:104A6A0082E4353DF58322E540255AF582E4353F57
:104A7A00F58322E56F256DF582E4356EF583E0FF57
:104A8A00E56F256DF582E4356EF58322E55A240239
:104A9A00FFE433FE22E56C2401FFE433FEC3E56D37
:104AAA009FEE6480F874809822EF2540FFEE353F30
:104ABA0022C2017FF47E01126BC9E56C25E0F56C18
:104ACA00756D0122E55C2EF582E4355BF583E0FD28
:084ADA0022753D1E753E6022AD
:106BC900EF1FAA0670011ED39400EA9400400BE45B
:0A6BD900FDEDC394C850E90D80F7EC
:016BE300228F
:105159008F5BE55BB401197D017F06124E3A500C55
:105169009000B1E0FF7C0D7D00125BCA78850622B4
:10517900E55BB402131251CB50439000B2E0FF7CBF
:105189000D7D20125BCA8035E55BB404161251CB44
:10519900500C9000B4E0FF7C0D7D60125BCA7885ED
:1051A900760622E55BB403197D027F06124E3A505A
:1051B9000C9000B3E0FF7C0D7D40125BCA788576C8
:0A51C90001227D027F06124E3A22F9
:104E3A00BF0107900020E0FE8048BF0207900021D2
:104E4A00E0FE803EBF0307900022E0FE8034BF04EC
:104E5A0007900023E0FE802ABF0507900024E0FEA9
:104E6A008020BF0607900025E0FE8016BF07079046
:104E7A000026E0FE800CBF0807900027E0FE8002B3
:104E8A00E4FEBD0103EE1322BD0204EEA2E122BD3F
:104E9A000304EEA2E222BD0404EEA2E322BD05044D
:104EAA00EEA2E422BD0604EEA2E522BD0704EEA2AC
:074EBA00E622BD0802EE3301
:014EC10022CE
:101E0B00124ADB900100E0F55A124A65E0123B8260
:101E1B001E3A011E6F021EA4031ED9041F0E051FBE
:101E2B0043061F78071FA8081FD40900001FFE12C6
:101E3B004A65A3E0B40A15E55A124A98E545B50779
:101E4B000BE4B506077D017F01021FBC124A59E561
:101E5B00456D7001EC6003021FFE124A4AC2287FD7
:101E6B0001021FD1124A65A3E0B40A15E55A124AC2
:101E7B0098E545B5070BE4B506077D017F02021F08
:101E8B00BC124A59E5456D7001EC6003021FFE124E
:101E9B004A4AC2287F02021FD1124A65A3E0B40A44
:101EAB0015E55A124A98E545B5070BE4B506077DCB
:101EBB00017F03021FBC124A59E5456D7001EC60AE
:101ECB0003021FFE124A4AC2287F03021FD1124A85
:101EDB0065A3E0B40A15E55A124A98E545B5070B18
:101EEB00E4B506077D017F04021FBC124A59E54584
:101EFB006D7001EC6003021FFE124A4AC2287F0478
:101F0B00021FD1124A65A3E0B40A15E55A124A988A
:101F1B00E545B5070BE4B506077D017F05021FBC40
:101F2B00124A59E5456D7001EC6003021FFE124A1F
:101F3B004AC2287F05021FD1124A65A3E0B40A15D5
:101F4B00E55A124A98E545B5070BE4B506077D013E
:101F5B007F06021FBC124A59E5456D7001EC600308
:101F6B00021FFE124A4AC2287F06021FD1124A657F
:101F7B00A3E0B40A14E55A124A98E545B5070AE4FA
:101F8B00B506067D017F078028124A59E5456D701D
:101F9B0001EC705F124A4AC2287F078029124A65FA
:101FAB00A3E0B40A0F124A65A3A3E070077D017F7B
:101FBB0008024DAF124A59E5456D7001EC703412B1
:101FCB004A4AC2287F080212F7124A65A3A3E0709F
:101FDB0022124A65A3E024F96008147016E4FF028C
:101FEB005ED97FF47E01126BC97D5E7F021266752E
:031FFB001242424D
:011FFE0022C0
:101C0A00753F1E7540B0900108E0F55A124A71E01E
:101C1A00123B821C3C011C74021CAC031CE4041D14
:101C2A001C051D54061D8C071DBF081DF409000064
:101C3A001E0A124A71A3E0B40A13124A96E546B57F
:101C4A00070BE4B506077D017F01021DD7AF5A12C3
:101C5A004A5BE5466D7001EC6003021E0A124AB344
:101C6A00124A51D2287F01021DF1124A71A3E0B42F
:101C7A000A13124A96E546B5070BE4B506077D0135
:101C8A007F02021DD7AF5A124A5BE5466D7001EC1E
:101C9A006003021E0A124AB3124A51D2287F020274
:101CAA001DF1124A71A3E0B40A13124A96E546B529
:101CBA00070BE4B506077D017F03021DD7AF5A1251
:101CCA004A5BE5466D7001EC6003021E0A124AB3D4
:101CDA00124A51D2287F03021DF1124A71A3E0B4BD
:101CEA000A13124A96E546B5070BE4B506077D01C5
:101CFA007F04021DD7AF5A124A5BE5466D7001ECAC
:101D0A006003021E0A124AB3124A51D2287F040201
:101D1A001DF1124A71A3E0B40A13124A96E546B5B8
:101D2A00070BE4B506077D017F05021DD7AF5A12DE
:101D3A004A5BE5466D7001EC6003021E0A124AB363
:101D4A00124A51D2287F05021DF1124A71A3E0B44A
:101D5A000A13124A96E546B5070BE4B506077D0154
:101D6A007F06021DD7AF5A124A5BE5466D7001EC39
:101D7A006003021E0A124AB3124A51D2287F06028F
:101D8A001DF1124A71A3E0B40A12124A96E546B549
:101D9A00070AE4B506067D017F078031AF5A124A69
:101DAA005BE5466D7001EC7057124AB3124A51D284
:101DBA00287F078032124A71A3E0B40A13124A96A6
:101DCA00E546B5070BE4B506077D017F08024DAF6E
:101DDA00AF5A124A5BE5466D7001EC7023124AB3A2
:101DEA00124A51D2287F080212F7124A71A3A3E0BD
:101DFA00700E124A71A3E024F870057F01125ED9B1
:011E0A0022B5
:0447C7008C5B8D5C1E
:1047CB00055CE55C7002055B14F5828C83E0F97087
:1047DB000302486EEF7005124ADB8009BF010675B4
:1047EB003F1E7540B0302846EF7007E96545600203
:1047FB00C322BF0107E965466002C322E4FEEEC394
:10480B00995029EF700F124ACEE53E2E124A69E0FD
:10481B006D6002C322EF6401700F124ACEE5402E89
:10482B00124A75E06D6002C3220E80D2D32220287B
:10483B0033E4FEEEC3995029EF700F124ACEE53EDA
:10484B002E124A69E06D6016C322EF6401700F12DD
:10485B004ACEE5402E124A75E06D6002C3220E80EF
:04486B00D2D322C3BF
:01486F002226
:0612F7008F5BAB05AA04A9
:1012FD007D027F07124E3A5011E55BB4050C8B82CF
:10130D008A83E0640570030215617D017F07124E2B
:10131D003A5011E55BB4050C8B828A83E06406704C
:10132D0003021561C229EB24FFF582EA34FFF58330
:10133D00E0F55D8B828A83E0FFF55EA3E0F9F55F52
:10134D00EF123B82136D01137402137B031382049E
:10135D00138905139006139707139E08000013A316
:10136D00755C01D229802F755C02D2298028755CAD
:10137D0004D2298021755C08D229801A755C10D29F
:10138D00298013755C20D229800C755C40D2298090
:10139D0005755C80D229E924FE700302146424F8DB
:1013AD00605C24096003021474E55BB401059000D0
:1013BD00208045E55BB40205900021803BE55BB4E0
:1013CD0003059000228031E55BB404059000238075
:1013DD0027E55BB40505900024801DE55BB406058B
:1013ED009000258013E55BB407059000268009E584
:1013FD005B64087074900027E0455CF0806BE55BE2
:10140D00B401059000208044E55BB40205900021F5
:10141D00803AE55BB403059000228030E55BB404AF
:10142D00059000238026E55BB40505900024801C03
:10143D00E55BB406059000258012E55BB4070590C9
:10144D0000268008E55BB40820900027E0FFE55CEE
:10145D00F4FEEF5EF08012E55BB4050B8B828A83A0
:10146D00E0FF123054C229C229202903021561E57B
:10147D005BB40109900020E0FD7F208060E55BB446
:10148D000209900021E0FD7F218052E55BB4030944
:10149D00900022E0FD7F228044E55BB404099000BA
:1014AD0023E0FD7F238036E55BB40509900024E041
:1014BD00FD7F248028E55BB40609900025E0FD7FC3
:1014CD0025801AE55BB40709900026E0FD7F268094
:1014DD000CE55BB4080C900027E0FD7F277E001221
:1014ED00636B126CDCD2AF2028047F0180027F0277
:1014FD00126E9AA228922F12692BAD5DE4FF12662F
:10150D0075AD5EE4FF126675E55FB401047D38804C
:10151D0007E55FB40A077D367F06126675E55BB495
:10152D0005031264CF7D077F05124E3A500A200045
:10153D0007C22F7F03122F1A7D017F01124E3A40F1
:10154D0005C22F122F1A7D017F02124E3A4005C29D
:04155D002F122F1A00
:011561002267
:024DAF008F5B18
:104DB100ED24FF922F12692BE55B123B824DDA0144
:104DC1004DDF024DE4034DE9044DEE054DF3064D73
:104DD100F8074DFD0800004E03900020802190004F
:104DE10021801C90002280179000238012900024C3
:104DF100800D90002580089000268003900027E018
:104E0100F55CE55C6024755E01E4F55DE55C30E030
:104E110007AD5EE4FF126675E55CC313F55C055EE4
:104E2100055DE55DC3940840E3227D187F021266AB
:084E3100757D537F02126675C6
:014E39002256
:1062C900C2AFD284C285BF070BC28600E580A2E2B5
:1062D90092298019BF080BC28600E580A2E39229A2
:1062E900800BBF0508C28600E580139229D286D2A9
:0562F90085D2AFA229CF
:0162FE00227D
:1043B600C228D22CE4FF1259A97D2E7F03126675FE
:1043C6007D607F021266757F03126E873023FD20A3
:1043D60023FDE5456407703B7E017F50124ADB8F63
:1043E600828E837407F07D01E53E2D124A69E582CF
:1043F60024FFF582E58334FFF583E0F9EF2DF5829E
:10440600E43EF583E9F00DBD08DED2287F647E0028
:10441600126BC97F081262C95043302895D22CE42A
:10442600FF1259A97D607F021266757D327F0612E2
:1044360066757D1E7F05126675C22CE4FF1259A9AA
:104446007C017D507B087F507E011254F57F081257
:1044560062C950097F327E00126BC980F07F647E8C
:0444660000126BC90C
:01446A00222F
:02548C008F5A35
:10548E00900138E0F55BE55A7020E55B124A98E52D
:10549E00456F7001EE704F7460255BF582E4341E2B
:1054AE00AF82F55D8F5E7F408024E55A64017036D1
:1054BE00E55B124A98E5466F7001EE702974B025CF
:1054CE005BF582E4341EAF82F55D8F5E7F101200B5
:1054DE0016855E82855D83E0FFA3E0FD126D408F31
:0654EE005CE4FD124EC259
:0154F4002295
:024EC2008D6BF6
:104EC40075F020EF900280123B76AF8285836E8F5F
:104ED4006FE0F56CD394004060E56C9410505AE593
:104EE4006B7014124ABD124A9F504E124A7D124FE3
:104EF40043056D056D80EFE56B64017019124ABBC3
:104F0400124A9F5034124A7D124F433023028029A3
:104F1400056D056D80EAE56B6402701D124ABB12D3
:104F24004A9F5015124A7DA3E0FD1264FF3023030B
:0E4F3400024F4A056D056D80E67F50126E53E8
:084F420022A3E0FD1264FF222E
:100D4200855C82855B83A3A3E0FF855C82855B83F0
:100D5200A3222430F58274003EF583EDF0AF62EFFA
:100D62003395E0FEE55F2FF582E55E3EF583A3A3B2
:100D7200E0FF126D1BAD07AF63EF3395E0FEEF228C
:100D8200A3A3E0FFE55C2404F582E4355BF583E090
:100D920022E55F2405F582E4355EF583E022E55F16
:100DA2002405F582E4355EF583E0FFE55F2406F570
:100DB20082E4355EF583E0222431F58274003EF54B
:100DC20083EDF0AF62EF3395E0FEE55F2FF582E54C
:100DD2005E3EF583222455F582E4340AF583EFF072
:100DE200E56275F007A422E562FD3395E0FCE55F5C
:100DF2002DF582E55E3CF583E0FFE55F2DF582E5AA
:100E02005E3CF583228E69F56AAF68EF3395E0FEAA
:100E1200E5662FF582E5653EF58322ECFF3395E02A
:100E2200FEEF25E0FFEE33FE75F020ED123B76E596
:100E3200822FF582E5833EF58322A3A3A3E0FF8DF3
:100E4200828C83E5822404F582E43583F58322E5EE
:100E5200662405F582E43565F583E022E55E75F0EA
:100E620007A42454F582E4340AF58322E55E75F082
:100E720007A42451F582E4340AF5832224E0F582A2
:100E8200740A3EF583E5822DF582E5833CF58322E3
:100E9200E55E75F007A42453F582E4340AF5832253
:100EA200E55F2405F582E4355EF583E0FFE55F2426
:100EB20006F582E4355EF583E022E55E75F007A46F
:100EC2002452F582E4340AF58322749F2562F58266
:100ED200E43400F58322746F2562F582E43400F570
:100EE20083222450F582E4340AF58322E560240546
:100EF200F582E4355FF58322D3EF6480948022ABE0
:100F020007AA068B828A83A3A3A3E0FFEB2404F53E
:100F120082E43AF583E0FD228F828E83A3A3A3E0CD
:100F220022855F82855E83A3A322AB5DAD5AAF5C4F
:100F3200AE5B2233CE33CE92E022A2E0CE13CE13AA
:100F42002275F00AA42DFDE5F03CFCE56622E56081
:100F52002405F582E4355FF583E022E56275F00849
:100F620090015822E55E75F007A42455F582E43419
:100F72000AF583E022AB5AAD5DAF5CAE5B22EF7C3B
:100F8200002563FDEC35628D82F58322A3A3E0FF89
:100F9200AD5A22E5662DF582E5653CF583A3A322D1
:100FA200540FF5657808AF03AE02EF08220564E539
:100FB20064AE632225E0FFEE33FE75F020E5642285
:100FC20075F020123B76E0FEA3E0FF22E0FAA3E0F8
:100FD200FB780CFFAE020822E0FCA3E0FD7804FFE0
:100FE200AE040822E5632561F582E43562F58322C9
:100FF200E5662DF582E5653CF58322E5662FF582EF
:10100200E5653EF583222480F58274023EAF82229A
:101012002560F560E4355FF55F22856082855F8338
:0B102200228F828E83A3A3E0640A22C9
:02055B008F5AB5
:10055D00C229E4F542D222D22C1259A97D4B7F0239
:10056D001266757D02E4FF1266757D32E4FF126638
:10057D00757D607F021266757D027F07124E3A50BF
:10058D00057F04126E87900528E0F536A3E0F53758
:10059D007F03126E87E55A7006A22392288009E523
:1005AD005AB40104A2249228E53745367005D229A4
:1005BD00020A223028DFE55A7006A223922880090C
:1005CD00E55AB40104A22492282028EAE55A700BBA
:1005DD00755B1E755C6085455D800EE55AB401093D
:1005ED00755B1E755CB085465DE55DD3940050036B
:1005FD00020A1C855C82855B83E0640B6003020A42
:10060D0017A3E0FFB40A0AE55DB40205D229020A78
:10061D001CEF6401701E120D4CA3E0640A7015E509
:10062D005D6405700F120D4C120D82120A4D1231C0
:10063D0082020A1C120D4CE0B40111120D4CA3E004
:10064D00B40109120F2C1217A9020A1C120D4CE04D
:10065D006401701E120D4CA3E064027015E55D641B
:10066D0005700F120D4C120D82120A4D1261780297
:10067D000A1C120D4CE06401701D120D4CA3E064B8
:10068D00037014E55DB4050F120D4C120D82FDAB18
:10069D005A1237EE020A1C120D4CE0B4011D120D58
:1006AD004CA3E0B40415E55DD39405400EAB5AADF3
:1006BD005CAC5BAF5D122CA1020A1C120D4CE06408
:1006CD0001701D120D4CA3E064057014E55DB405B9
:1006DD000F120D4C120D82FDAB5A125A9B020A1CC1
:1006ED00120D4CE06401701D120D4CA3E0640670F8
:1006FD0014E55DB4050F120D4C120D82FDAB5A12AF
:10070D004D22020A1C120D4CE0B4011D120D4CA31A
:10071D00E0B40715E55DD39405400EAB5AAD5CAC66
:10072D005BAF5D124300020A1C120D4CE0640170B8
:10073D001D120D4CA3E064087014E55DB4050F1295
:10074D000D4C120D82FDAB5A126335020A1C120DAF
:10075D004CE0B40215120D4CA3E0B40A0DE55DB4E6
:10076D000308AF5A1262FF020A1C120D4CE0B402CC
:10077D0016120D4CA3E0B4010EE55DB40E09120F77
:10078D002E122DDE020A1C120D4CE0B40216120DB3
:10079D004CA3E0B4020EE55DB40709120F2E125200
:1007AD00C6020A1C120D4CE0B40215120D4CA3E04A
:1007BD00B4090DE55DB40308AF5A125420020A1CAA
:1007CD00120D4CE064027019120D4CA3E0B4091126
:1007DD00E55DB4040C120D4C120F8E12671B020A4C
:1007ED001C120D4CE064037021120D4CA3E0640A41
:1007FD007018E55D64057012120D4C120D82FD121C
:10080D006D40AD5A124671020A1C120D4CE0640384
:10081D007029120D4CA3E064017020E55DD39405A1
:10082D004019120D4C120D82FD126D40855A62ABAE
:10083D005DAD5CAC5B123D6A020A1C120D4CE064AE
:10084D00037021120D4CA3E064027018E55D640580
:10085D007012120D4C120D82FD126D40AD5A125FC9
:10086D0059020A1C120D4CE0B40315120D4CA3E0F5
:10087D00B4030DE55DB40308AF5A125FD5020A1C2F
:10088D00120D4CE0B40318120D4CA3E0B40410E5A6
:10089D005DD394034009120F771249B1020A1C125D
:1008AD000D4CE0B40315120D4CA3E0B4050DE55D40
:1008BD00B40308AF5A126D2E020A1C120D4CE0B48F
:1008CD000316120D4CA3E0B4060EE55DB405091236
:1008DD000F2E12682A020A1C120D4CE064037019C7
:1008ED00120D4CA3E0B40711E55DB4040C120D4CD0
:1008FD00120F8E126B39020A1C120D4CE0B4031646
:10090D00120D4CA3E0B4080EE55DB40409120F2ED0
:10091D0012684F020A1C120D4CE064057014E55D5F
:10092D00B4040F120D42A3A3E0FDAB5A121FFF0238
:10093D000A1C120D4CE0B40516120D86B40B10E511
:10094D005DD394054009120F771233DB020A1C1296
:10095D000D4CE064067014E55DB4040F120D42A356
:10096D00A3E0FDAB5A1221F1020A1C120D4CE0B4AA
:10097D000616120D86B40B10E55DD39405400912D1
:10098D000F77122719020A1C120D4CE06409701A18
:10099D00120D4CA3E0B40A12E55DB4040D120D4C1A
:1009AD00A3A3E0FF125D86020A1C120D4CE0640940
:1009BD007018120D4CA3E0B40110E55DB4040B12D8
:1009CD000D4C120F8E12625B8045120D4CE0B40976
:1009DD0017120D4CA3E0B4020FE55DD3940440084B
:1009ED00120F2C1215628027120D4CE06409701A3B
:1009FD00120D4CA3E0B40310E55DB4040B120D4CC5
:100A0D00120F8E125CF480078000AF5A126B5620C5
:100A1D0029030205A2C21DD22CAF5A1259A97D601D
:100A2D007F021266757D327F031266757F03126E2B
:0F0A3D0087125DCE7FFF126E53E47885F6C222DA
:080A4C0022FD126D40AD5A229B
:0817A9008E5E8F5F8D608B6185
:1017B100120F1AFFE55F2404120D97FD12640A8FC0
:1017C1006274E22562F562C3940050030219AAE52E
:1017D10062941440030219AAE5616406701D120D9A
:1017E10093B4010C120DE2120EE47401F00219A679
:1017F100120DE2120EE4E4F00219A6E561640E6036
:10180100030218C8E55F240C120D97FFB40A14E512
:101811005F240D120D97B40A0A120DE2120E74E440
:10182100F08013E55F240D120D97FD126BAD120DC3
:10183100E2120E74EFF0E55F240A120D97FFB40A6D
:1018410014E55F240B120D97B40A0A120DE2120E71
:10185100C2E4F08013E55F240B120D97FD126BAD0E
:10186100120DE2120EC2EFF0E55F2409120D97FF8F
:10187100640A6006EFD39409400A120DE2120E9831
:10188100E4F08010E55F2409120D97FF120DE212BA
:101891000E98EFF0120D93FFB40B15E55F240612BD
:1018A1000D97B40B0B120DE2120E6474FFF0800859
:1018B1001219D6120E64EFF01219B2120DD7120ED0
:1018C100E47401F00219A6E561640A706E120DE27A
:1018D100120E74E4120DE1120EC2E4F0E55F240968
:1018E100120D97FF640A6006EFD39409400A120DA6
:1018F100E2120E98E4F08010E55F2409120D97FFC3
:10190100120DE2120E98EFF0120D93FFB40B15E5D4
:101911005F2406120D97B40B0B120DE2120E6474C4
:10192100FFF080081219D6120E64EFF01219B212EC
:101931000DD7120EE47401F00219A6E56164097075
:1019410068120DE2120E74E4120DE1120EC2E412DD
:101951000DE1120E98E4F0120D93FFB40B15E55F43
:101961002406120D97B40B0B120DE2120E6474FFD4
:10197100F08013E55F2406120D97FD126BAD120D79
:10198100E2120E64EFF0E55F2407120D97FFE55FA9
:101991002408120D97FD126BAD120DE2120DD71234
:1019A1000EE47401F0D22B8002C22BAF60126E29BB
:1019B10022E55F2407F582E4355EF583E0FFE55F0C
:1019C1002408F582E4355EF583E0FD126BADE56236
:1019D10075F007A422E55F2406F582E4355EF58300
:0C19E100E0FD126BADE56275F007A4227A
:103182008F5E8D5FE55ED3941D500302328EE55E45
:103192009432400302328ED22CAF5F1259A97D467F
:1031A2007F07126675AF5E12350374E2255EF55E27
:1031B200120E70E07021120EBCE0701B120E92E033
:1031C2007015120E5EE0700F120F66700A1232A7AF
:1031D2007D537F02023284123296E55E75F007A4B7
:1031E200120EE4E070047D3680027D387F0612669E
:1031F20075123296120E6EE0FFD394014034EF94B2
:1032020013502F7D097F06126675120E6E12329EC2
:103212007FF47E01126BC97D0E7F031266757D35C8
:103222007F061266757D097F06126675120EBC1244
:10323200329E7FF47E01126BC9120E92E0FF60058E
:10324200125A4C800A1232A77D0F7F031266757DD7
:10325200277F02126675120E5EE0FFF46008126CA0
:103262004E12350380077D187F021266757D377F07
:1032720004126675120F66FF126C4E1235037D053D
:103282007F06126675C22CAF5F0259A9C22BAF5FCF
:10329200126E29227FF47E01126BC922E0FF126CAA
:0D32A2004E123503227D187F021266752240
:026178008D5E3A
:10617A00EFD3941D402AEF9432502574E22FFFE4A6
:10618A00FEEEFD3395E0FCEF75F007A42450F5828E
:10619A00E4340A120E85E4F00EBE07E5D22B800223
:0761AA00C22BAF5E126E294B
:0161B10022CB
:062DDE008E5E8F5F8D6028
:102DE400D22A120F1AFFE55F2404120DB1122F0527
:102DF400C39418501C855F82855E83A3A3A3E0FF60
:102E0400E55F2404120DB1FD126D087883A60780D6
:102E140006E47883F6C22A120DA0122F05C3943C4F
:102E2400500D120DA0FD126D087884A6078006E4EB
:102E34007884F6C22AE55F2407120DB1FF126DBB38
:102E44008F61E561D394004017E56194085011E562
:102E54005F2407120DB1FF126DBB7880A6078006B0
:102E640078807601C22AE55F2408120DB1FFE55F80
:102E74002409120DB1122F0E401FE5619420501940
:102E8400E55F2408120DB1FFE55F2409120DB1FDC1
:102E9400126D087888A607800678887601C22AE52C
:102EA4005F240A120DB1FFE55F240B120DB1122F3E
:102EB4000E401FE561940D5019E55F240A120DB10F
:102EC400FFE55F240B120DB1FD126D087881A60792
:102ED400800678817601C22AE55F240C120DB1FFC9
:102EE400E55F240D120DB1FD126D087882A607303E
:102EF4002A07125795D22B8002C22BAF60126E297B
:102F040022FD12640A8F61E56122FD12640A8F6159
:062F1400E561D3940022E8
:0652C6008E5E8F5F8D601B
:1052CC00D22A120F1AFFE55F2404120EB3125331C7
:1052DC009418501C855F82855E83A3A3A3E0FFE531
:1052EC005F2404120EB3FD126D087883A6078006A6
:1052FC00E47883F6C22A120EA2125331943C500D5C
:10530C00120EA2FD126D087884A6078006E478843C
:10531C00F6C22A302A07125795D22B8002C22BAF25
:04532C0060126E2974
:0B53300022FD12640A8F61E561C322B8
:106DBB00120EFA4008EF6480948A5001227F002261
:106D0800AE05126DBBEFC454F0FDAF06126DBBEFBC
:036D18004DFF220A
:1062FF008F5ED22C1259A97D1E7F081266757D26DE
:10630F007F081266757D527F04126675C22A126865
:10631F0004125C607880E6FF125A4C125953C22C5B
:06632F00AF5E1259A92225
:10671B008D5EEFD3940A4006EFD3940F4003EF70D6
:10672B000E90002BEFF0D22BAF5E126E29D322C24C
:08673B002BAF5E126E29C32290
:025420008F5E9D
:10542200D22C1259A97D207F051266757D2E7F032D
:105432001266757D527F0412667590002BE0F55F4F
:10544200E55FB40B067D5F7F078034E55FB40C0631
:105452007D5E7F068029E55FB40D067D0A7F0280AE
:105462001EE55FB40E067D327F028013E55FB40F46
:10547200067D467F028008E55F70077D0A7F031282
:095482006675C22CAF5E1259A937
:01548B0022FE
:106B39008D5E120EFA400EEF648094865007126340
:0D6B4900D6D22B8002C22BAF5E126E292225
:02682A008D5E81
:10682C00120F0112640A120EFA4010EF648094A148
:10683C005009900029EFF0D22B8002C22BAF5E12D0
:02684C006E29B3
:01684E002227
:02684F008D5E5C
:10685100120F0112640A120EFA4010EF648094A123
:106861005009900028EFF0D22B8002C22BAF5E12AC
:026871006E298E
:016873002202
:106D1B00D3EF648094814008EF6480948950012202
:036D2B007F0022C4
:106DCB00120EFA4008EF648094A15001227F00223A
:081562008E5E8F5F8D608B61CE
:10156A00120F1A14F56374FC2561F5616403600FA8
:10157A00E56164076009E561640B6003021744C30F
:10158A00E563648094805003021744E563648094A1
:10159A00884003021744E4F562120D797803C333D5
:1015AA00CE33CED8F92430F58274003EF583AF628B
:1015BA00EF3395E0FE120E31E4F00562E562B408FD
:1015CA00D8756204E56164037027120DE912179F4A
:1015DA00120D777803C333CE33CED8F9120D54786F
:1015EA0003C333CE33CED8F92431F58274000217FF
:1015FA003BE5616407705D120DE912179F120D77C2
:10160A007803C333CE33CED8F9120D547803C333DB
:10161A00CE33CED8F9120DBAA3120D707803C333A4
:10162A00CE33CED8F912174CC333CE33CED8F924E1
:10163A0033F5827400120DC0E5822406120E491297
:10164A000D727803C333CE33CED8F92434F58274BD
:10165A000002173BE561640B6003021744120DE9AF
:10166A00A3E0FD12640A126DCB120D777803C3331F
:10167A00CE33CED8F9120D547803C333CE33CED835
:10168A00F9120DBAA3120D707803C333CE33CED834
:10169A00F912174CC333CE33CED8F92433F58274FA
:1016AA0000120DC0E5822406120E49120D7278034B
:1016BA00C333CE33CED8F92434F5827400120DC068
:1016CA00E5822407120E49120D727803C333CE3312
:1016DA00CED8F92435F58274003EF583EDF0E56243
:1016EA00FD3395E0FC120DFCE5822408F582E43511
:1016FA0083120DF8E5822409120E49E0FD12640AEC
:10170A00126DCB120D777803C333CE33CED8F924BA
:10171A0036F5827400120DC0E582240A120E4912AF
:10172A000D727803C333CE33CED8F92437F58274D9
:10173A00003EF583EDF0D22B8002C22BAF60126E11
:01174A002975
:10174B00222432F58274003EF583EDF0E562FD3321
:10175B0095E0FCE55F2DF582E55E3CF583E58224A3
:10176B0004F582E43583F583E0FFE55F2DF582E533
:10177B005E3CF583E5822405F582E43583F583E051
:10178B00FD12640A126DCBAD07AF63EF3395E0FE2C
:0E179B00EF780322A3E0FD12640A126DCB2248
:045CF4008D5EAC070E
:105CF800D3EC648094804035EC64809489502EE421
:105D0800FDECFF3395E0FEEF7803C333CE33CED8F6
:105D1800F92428F58274003EF583EDFF3395E0FE03
:105D2800120E31E4F00DBD08D8D22B8002C22BAF81
:045D38005E126E2960
:015D3C002244
:10625B008D5E120EFA402FEF648094895028EF1454
:10626B00FFE55E24FF922A124FD2D22CAF5E125959
:10627B00A97542017F327E00126BC9E54270FCC2E8
:07628B002CAF5E1259A9229D
:084300008F5E8C5F8D608B6104
:10430800856082855F83120E3CE0FD12640A8F622D
:10431800E562D3940050030243AEE5629432400351
:104328000243AEE55E64067036D22CAF611259A91D
:104338007D527F05126675AF62123503120F50B4B5
:10434800010A120ECC7401F07D388007120ECCE4FD
:10435800F07D367F06126675C22CAF610259A9E559
:10436800602406120F54640B703C120F50B40108FD
:10437800120ECC7401F08005120ECCE4F074F9250D
:104388005EF55E75F004123ABCAFF0EF7014E560AC
:104398002406FBE4355FFAAD62E4FF1236F9D22B4E
:0D43A8008006C22B8002C22BAF61126E296D
:0143B50022E5
:082CA1008F5E8C5F8D608B617A
:102CA900856082855F83120E3CE0FD12640A8F62A3
:102CB900E562D394005003022DD6E56294284003BF
:102CC900022DD6E55E64067037D22CAF611259A980
:102CD9007D527F05126675AF62123503120EEEE062
:102CE900B4010A120ED87401F07D388007120ED88B
:102CF900E4F07D367F06126675C22CAF610259A9D0
:102D0900E5602406120EF2E0640B6003022DD61270
:102D19000EEEE0B40108120ED87401F08005120E0F
:102D2900D8E4F0E4FFFEE5602407120EF2E5822EF6
:102D3900120E49E0B40B04AF0680040EBE08E7EF9B
:102D49007003022DD6C394084003022DD6120F5DDD
:102D5900123B76EFF07E01EF2401FDE433FCEEC374
:102D69009DEC6480F87480985020E5602406120E6A
:102D7900F2E5822E120E49E0FD120F5D123B76E557
:102D8900822E120E49EDF00E80CDE5602408120E58
:102D9900F2E5822F120E49E0640B602DEF2408FE44
:102DA900C3E55E9EF55E75F004123ABCAEF0EE70B6
:102DB9001CE5602407FDE4355FFC7E00ED2FFBEE8A
:102DC9003CFAAD627F011236F9D22B8002C22BAFD9
:042DD90061126E29EC
:012DDD0022D3
:0836F9008F638D648A658B6606
:10370100756801E4F567120E0BE0FF64097037126A
:1037110037DF8003120F35D8FB120E071237D1782D
:1037210008EF088003120F35D8FB8E69F56AE5684A
:10373100FD3395E0FC120F95E0FF120F95A3E0FD1C
:10374100126D4002378E120E0BE0FF1237DF80033D
:10375100120F35D8FB120E071237D17804EF08800B
:1037610003120F35D8FB120E07A3A3E0FF126E7DE3
:10377100EF426AAE69AF6A7804EF088003120F3531
:10378100D8FB120E07A3A3A3E0FF126E7DEF426ADE
:10379100E563700DAF67120D7B120FB6900AC08002
:1037A10010E563B40115AF67120D7B120FB69005DA
:1037B10030120E2EE569F0A3E56AF074042568F570
:0F37C100680567C3E5676480949050030237077B
:1037D00022A3E0FF126E7DEF426AAE69AF6A221249
:0E37E0006E7D7569008F6AAE697804EF08226D
:0A6E7D00EFD3940940037F002222A6
:0237EE008B5EF0
:1037F00012640A8F61E561D3940050030238D7E563
:1038000061943340030238D7D22CAF5E1259A97DA0
:10381000527F05126675AF61123503746F25611210
:103820000EDCE060047D3880027D367F061266750E
:103830007F2C7E01126BC9E561120F5F123B76E0AF
:10384000F55F70077D1B7F061266757D577F02123C
:103850006675E55F603F756001AF5F120D7B240107
:10386000FFE43EFEAD60ED3395E0FCC3ED9FEE64FA
:1038700080F8EC648098501DAF60EF3395E0FE75E2
:10388000F008E561900158120E2EE0FDE4FF12668B
:1038900075056080C47F2C7E01126BC9E5619005BF
:1038A00030120FC2900000EEF0A3EFF04E70077DD3
:1038B0001B7F061266757D0C7F03126675900000F3
:1038C000E07002A3E06009E56114FD7F01122A03A4
:0E38D000C22CAF5E0259A9C22BAF5E126E2948
:0138DE0022C7
:024D22008B5EA6
:104D240012640A8F5FE55FD394004077E55F9433A4
:104D34005071D22CAF5E1259A97D527F051266754F
:104D4400AF5F123503749F255F120ED0E060047DBF
:104D54003880027D367F061266757F2C7E01126BC9
:104D6400C97F2C7E01126BC9E55F900AC0120FC285
:104D7400900000EEF0A3EFF04E70077D1B7F06124B
:104D840066757D0C7F03126675900000E07002A3C7
:104D9400E06009E55F14FDE4FF122A03C22CAF5E54
:0A4DA4000259A9C22BAF5E126E295E
:014DAE0022E2
:026335008B5E7D
:1063370012640AAD07EDD394004021ED9433501C4D
:10634700E4FC900AC0120E1DE4F0A3F00CBC10F29E
:10635700749F2D120ED0E4F0D22B8002C22BAF5EB9
:03636700126E298A
:01636A002210
:025A9B008B5E20
:105A9D0012640AAD07EDD394004038ED94335033C2
:105AAD00E4FC900530120E1DE4F0A3F00CBC10F2D6
:105ABD00746F2D120EDCE4F0FCECFF3395E0FE75F7
:105ACD00F008ED900158120E2EE4F00CBC08EAD24D
:0A5ADD002B8002C22BAF5E126E296F
:015AE700229C
:042A03008F628D63EE
:102A0700E4F564E5627052AF64120D7B25E0FDEEDC
:102A170033FCAF63120D7B7805C333CE33CED8F9C1
:102A2700120E7E120FCE8003120F3CD8FB120FA29C
:102A37008003120F3CD8FB540FF566AF63120D7B72
:102A47007805C333CE33CED8F9120E7E120FDA8053
:102A570003120F3CD8FB022AC1E56264017064AF20
:102A670064120D7B25E0FDEE33FCAF63120D7B781E
:102A770005C333CE33CED8F92450F5827405120E30
:102A870084120FCE8003120F3CD8FB120FA28003D3
:102A9700120F3CD8FB540FF566AF63120D7B780518
:102AA700C333CE33CED8F92450F5827405120E8481
:102AB700120FDA8003120F3CD8FB540FF567ED5461
:102AC7000FF568E565700CE5667008E5677004E565
:102AD70068607CAD65E4FF126675AD66E4FF12665B
:102AE70075E56564097045856769AF69FE7804EF28
:102AF700088003120F35D8FBF569E5684269E56977
:102B0700B4990B7D09E4FF1266757D098027E56995
:102B170075F00A84F56AFDE4FF126675E56A75F0DB
:102B27000AA4FFC3E5699FF56AFD8009AD67E4FF65
:102B3700126675AD68E4FF1266757FF47E01126B4D
:0F2B4700C90564C3E564648094A05003022A0AA0
:012B5600225C
:10640A00EFD394004015EF940B5010EFC3940A5049
:10641A0008EF75F00AA4FE8002E4FEEDD394004072
:10642A000EED940B5009EDC3940A5003ED2EFEAF06
:01643A00065B
:01643B00223E
:0649B1008E5E8F5F8B603B
:1049B700756105756240D3ED64809484407CED6435
:1049C7008094A55075ED24FDF563D39404406BE501
:1049D7006320E06613F5640562E562AE6170020567
:1049E7006114F5828E83E564F07403255FF55FE457
:1049F700355EF55EE4F563E563C395645033855F23
:104A070082855E83E0FFA3E0FD126D400562E562EB
:104A1700AC617002056114F5828C83EFF0055FE5E8
:104A27005F7002055E055FE55F7002055E056380E6
:104A3700C6D22BAF60126E29D322C22BAF60126E83
:024A470029C381
:014A4900224A
:043D6A008C5F8D607D
:103D6E00120EFA5003023E42EF6480949540030215
:103D7E003E42EB648094875003023E42EB64809493
:103D8E00E44003023E42120D7B7805C333CE33CEA0
:103D9E00D8F9121008F5638F64EB24FBF565D39404
:103DAE00025003023E42E56575F00384E5F06003C0
:103DBE00023E42E56575F00384F567C394105074B6
:103DCE00120FAF7002056314F5828E83E567F074EF
:103DDE0005121012E4F565E565C395675052121091
:103DEE001CE0F566B40A10120FAF7002056314F5ED
:103DFE00828E83E4F0800F120FAF7002056314F50C
:103E0E00828E83E566F012101CA3E0FF12101CA335
:103E1E00A3E0FD126D408F66120FAF7002056314A2
:103E2E00F5828E83E566F07403121012056580A785
:0B3E3E00D22B8002C22BAF62126E2953
:013E49002256
:082719008E5E8F5F8D608B6105
:10272100C22A12102360030227B612289150030215
:1027310027B1E5649408E56394075074C3E56064C8
:1027410080948A506B120F23A3E0F562B4010690C6
:102751000520022806E562B4020690052202280639
:10276100E562B40306900524022806E562B4040676
:10277100900526022806E562B40506900528022880
:1027810006E562B4060690052A022806E562B4074A
:102791000690052C022806E562B4080590052E80F6
:1027A10064E562B40905900530805AD22A02288274
:1027B100D22A022882120F23E064017052AD60AF69
:1027C1005FAE5E1228915003022882E5649408E509
:1027D1006394074003022882C3E5606480948A40C1
:1027E10003022882120F23A3E0F562B40A059005C3
:1027F100328012E562B401059005348008E562B4C7
:102801000209900536E563F0A3806FD22A80721227
:102811000F23E06402706AAD60AF5FAE5E125B349D
:102821007563008F64C3E5649463E563940050515C
:10283100C3E560648094885048120F23A3E0F562D9
:10284100B40107900538EFF08037E562B4020590D6
:1028510005398026E562B4030590053A801CE562DE
:10286100B4040590053B8012E562B4050590053C72
:102871008008E562B4060890053DE564F08002D267
:0F2881002A302A04C22B8002D22BAF61126E299B
:10289000221248708E638F64D3E564943BE56394A1
:0228A000002214
:064870008E658F66A905AC
:104876007D057C00120FF2E0C3940A4005120FF288
:10488600E4F00DBD00010CED640A4C70E7B90607B3
:10489600120E51FF7E0022E964077010120E517548
:1048A600F00AA4ACF0FDE5662406801BE9640870F6
:1048B60021120E5175F064A4ACF0FDE566240612D3
:1048C6000E55120F432407120E552DFDE43CAF057D
:1048D600FE22E964097033120E51FF7E007C037DCF
:1048E600E8123ADEAC06AD07E5662406120E5575EB
:1048F600F064120F462407120E55120F43240812B5
:0D4906000E552DFDE43CFEAF0522E4FEFF42
:014913002281
:065B34008E658F66A905D5
:105B3A007F057E00120FFDE0C3940A4005120FFD97
:105B4A00E4F00FBF00010EEF64084E70E7E9640746
:105B5A007020E5662405F582E43565F583E075F085
:105B6A000AA4FFE5662406F582E43565F583E02F8D
:045B7A00FF227F0087
:015B7E002204
:0833DB008E5E8F5F8D608B6137
:1033E300C22AD3E560648094845003023489E56083
:1033F3006480948D400302348912102360030234E5
:1034030089120F1A123B82342901343402343F03E8
:10341300344904345305345D063467073471083482
:103423007B0900003485756201756300D22A02347A
:10343300C0756201756308D22A0234C075620175D2
:103443006310D22A8077756201756318D22A806D62
:10345300756201756320D22A8063756201756328E2
:10346300D22A8059756201756330D22A804F756202
:1034730001756338D22A8045756201756340D22A8B
:10348300803BC22A8037D3E56064809484402EE574
:10349300606480948D5026855F82855E83A3A3E05C
:1034A300B4011A855F82855E83A3A3A3E024F6702B
:1034B3000A756201756358D22A8002C22A302A38FB
:1034C300E4FF120F80E4F00FBF08F7E56024FB85EB
:1034D3006382856283F07F01E55F2404F582E4352E
:1034E3005EF583E5822F120E49E0FE120F80EEF0A7
:0F34F3000FBF08E4D22B8002C22BAF61126E29EB
:0135020022A6
:044671008F5E8D5F6C
:10467500E55ED394005003024714E55E94154003AC
:10468500024714D22CAF5F1259A97D5F7F051266D0
:1046950075AD5EE4FF1266757D527F041266757F07
:1046A500F47E01126BC975F020E55E900280123B25
:1046B50076AF828583628F63E0F560603DD39400B9
:1046C5004046E56094105040E56025E0F560756171
:1046D50001E5602401FFE433FEC3E5619FEE6480DC
:1046E500F87480985022120FE6E0FF120FE6A3E05F
:1046F500FD1264FF0561056180D77D1B7F0612668B
:10470500757D5F7F05126675C22CAF5F0259A9C220
:064715002BAF5F126E29BC
:01471B00227B
:1021F1008F5E8D5F8B60E55E640A7074E55FC394EA
:102201000A400302235E122394E4FDFF126675ADBA
:102211005F12236DE55F123B82223901223F0222C8
:102221004503224B04225105225706225D072263F2
:10223100082269090000226E9005200222B890054B
:10224100220222B89005240222B89005260222B863
:102251009005280222B890052A0222B890052C0286
:1022610022B890052E0222B8900530804A022357E9
:10227100E55E64017052E55FD394004006E55F942A
:10228100034006E55F640A703C122394E55FB40ADB
:102291000A7D0A12236D900532801CE55FB4010AA4
:1022A1007D0B12237A900534800DE55FB402137D16
:1022B1000C12237A900536E0FEA3E0FF12646E0251
:1022C100236502235702235EE55E64026003022355
:1022D10065E55FD39400500302235EE55F940750E8
:1022E1007CD22CAF601259A97D277F081266757DBB
:1022F10006E4FF1266757D14E4FF126675E55F243E
:10230100FE601A14602114602814602F14603624B2
:102311000570437D0112238790053880307D0212BC
:10232100238790053980267D031223AA90053A80E0
:102331001C7D041223AA90053B80127D051223B750
:1023410090053C80087D061223B790053DE0FF7E95
:102351000012649F800EAF60126B568007C22BAFD4
:1023610060126E29C22CAF601259A922E4FF1266D5
:10237100757D527F0412667522E4FF1266757D52E7
:102381007F0412667522E4FF1266757D527F041286
:10239100667522D22CAF601259A97D277F0812667B
:1023A100757D06E4FF12667522E4FF1266757D52A3
:1023B1007F0412667522E4FF1266757D527F041256
:0323C1006675221C
:044AE2008E638F64EC
:104AE6000564E5647002056314F5828E83E0F5665D
:104AF600607AC3940850757F2C7E01126BC9E4F569
:104B060065E565C395665064856482856383E012B6
:104B16003B824B53004B310A4B350B4B3B0C4B4105
:104B26000D4B470E4B4D0F00004B59E4FD802D7D7C
:104B36005F7F0780287D5E7F0680227D0A7F028058
:104B46001C7D327F0280167D467F0280107D0A7FA3
:104B560003800A856482856383E0FDE4FF1266753F
:0C4B66000564E564700205630565809538
:014B72002220
:061FFF008F5E8D5F8B6018
:10200500C22AE55E640A60030220F3E55F123B82A3
:10201500203401204702205A03206D04208005202A
:10202500960620AC0720C20820D709000020EF1231
:1020350021287D01122176756101756200D22A027F
:10204500210F1221287D0212217675610175620822
:10205500D22A02210F1221447D03122183756101C9
:10206500756210D22A02210F1221447D04122183A8
:10207500756101756218D22A02210F1221601221A1
:10208500D67D051221A6756101756220D22A02212D
:102095000F1221601221D67D061221A675610175E8
:1020A5006228D22A02210F1221901221EA7D0712FD
:1020B50021B3756101756230D22A02210F12219078
:1020C5001221EA7D081221B3756101756238D22AA1
:1020D50080381221C0E4FDFF1266757D091221DDED
:1020E500756101756240D22A8020C22A801CE55E96
:1020F50064017016E55F24F670101221C07D0A1286
:1021050021DD756101756258D22A302A09AF62AEA8
:1021150061124AE28005AF60126B56C22CAF6012A5
:0221250059A9B6
:1021270022D22CAF601259A97D577F021266757DA6
:1021370005E4FF126675E4FDFF12667522D22CAF27
:10214700601259A97D577F021266757D05E4FF125B
:102157006675E4FDFF12667522D22CAF601259A98D
:102167007D577F021266757D05E4FF12667522E4CE
:10217700FF1266757D527F0412667522E4FF1266B0
:10218700757D527F0412667522D22CAF601259A951
:102197007D577F021266757D05E4FF12667522E49E
:1021A700FF1266757D527F0412667522E4FF126680
:1021B700757D527F0412667522D22CAF601259A921
:1021C7007D577F021266757D05E4FF12667522E46E
:1021D700FDFF12667522E4FF1266757D527F0412B9
:0A21E700667522E4FDFF1266752202
:103503008F72E572D3945940107D5A1235EA24A67E
:10351300FD70030235E90235E4E572D3944F40169A
:10352300E572945A50107D501235EA24B0FD7003B1
:103533000235E90235E4E572D394454016E5729409
:103543005050107D461235F224BAFD70030235E95E
:103553000235E4E572D3943B4012E5729446500C75
:103563007D3C1235F224C4FD607C8075E572D394F2
:10357300314012E572943C500C7D321235FA24CE60
:10358300FD6063805CE572D394274012E572943248
:10359300500C7D281235FA24D8FD604A8043E57229
:1035A300D3941D4016E572942850107D1EE4FF123B
:1035B3006675E57224E2FD602D8026E572D39413CF
:1035C3004016E572941E50107D14E4FF126675E5F3
:1035D3007224ECFD60108009E572C394145007ADAA
:1035E30072E4FF12667522E4FF126675E57222E447
:0F35F300FF126675E57222E4FF126675E572221B
:1059A9008F6AE56A700C302C097F01126E9A7FC0EC
:1059B900801FE56A700C202C097F01126E877FC059
:1059C9008026E56AB40112302C0F7F02126E9A7F8D
:1059D90030120016C22F02692BE56AB40114202C7B
:1059E900117F02126E877F30126E537FC87E0012BC
:0359F9006BC92255
:106907008F69D22C1259A97D607F021266757D327C
:106917007F061266757D1E7F05126675C22CAF69EC
:046927001259A92236
:106B56008F69D22C1259A97D607F021266757D302D
:0D6B66007F03126675C22CAF691259A92277
:0E6E29008F68302B03026907AF68126B562288
:105D8600EF24FE60101460162402701C7F01126E50
:105D96009A7F8080107F02126E9A7F2080077F0391
:105DA600126E9A7FA01200167FF47E01126BC975DF
:105DB6004204E54270FC7F647E00126BC97F0312C9
:085DC6006E877FA0126E5322CC
:10649F008E618F627C007D0A123AF0AD07E4FF1225
:1064AF0066757D5B7F06126675AE61AF627C007D9F
:1064BF000A123AF0E4FF1266757D4A7F070266758D
:04646E008E618F624A
:106472007C007D3C123AF01235037D057F061266E0
:1064820075AE61AF627C007D3C123AF0ED4C600C5F
:0C649200AF051235037D4A7F07126675C6
:01649E0022DB
:025F59008D5E5B
:105F5B00120EFA402FEF648094955028120D7B7827
:105F6B0005C333CE33CED8F9121008FEE4FD0FEF84
:105F7B00AA0670010E14F5828A83E4F00DBD20EEA3
:0B5F8B00D22B8002C22BAF5E126E29E9
:015F960022E8
:105FD5008F5E900540E0D394024015D22C1259A94A
:105FE5007542037F327E00126BC9E54270FC801555
:105FF500D22CAF5E1259A97D1B7F061266757D0CEA
:0D6005007F03126675C22CAF5E1259A922EE
:106D2E007E10900540E4F0A3DEFC7E10D22B126E96
:016D3E00292B
:016D3F002231
:106D4000BF0A02E4FFBD0A02E4FDEF75F00AA42DBC
:026D5000FF2220
:106BAD00EFD394094002E4FFEDD394094002E4FDD4
:0C6BBD007804EF08800123D8FD4DFF2272
:103FF7000701020304050607070706050403020174
:1040070003010A0A030307050303020503020A0A59
:1040170004050A0A0104050A0A0A04050A0A020332
:10402700070A0A03040A0A04024B00020032072E99
:1040370003024B0002003202055F000302055F0026
:104047000402055F000502055F000604072E082627
:104057000640033204072E08260640025304081EB2
:1040670008260452010008024B00020032072E08FE
:104077001E08260452010003072B023506360307E4
:104087002B0235063803072B0235072603072B02B9
:1040970035025302055F000F02055F001002055F3E
:1040A700001102055F001202055F001302055F00A1
:0A40B70014080C0A1D020500241B6A
:10524D007461F0A37420F0A37452F0A37401F0A361
:10525D0022A3F0A37461F0A37440F022F0A37403B1
:10526D00F0E4A3F0A37410F0A37403F0E4A3F0A38F
:10527D00227461F0A37441F0A3227461F0A3F0A332
:10528D007430F0A3227496F0A37432F0A37495F0E9
:10529D00A3741EF0A322F0A37461F0A314F0A37401
:1052AD0070F0A3E4F022A3F0A37452F0A3223CF516
:0952BD0083E0FEEF3395E0FC22D2
:10003E007E3F7FF77C017D507B081260C77E3F7F3D
:10004E00FF7C017D587B081260C77E407F077C01D4
:10005E007D007B041260C77E407F137C017D087B90
:10006E00041260C77E407F0F7C017D107B041260FE
:10007E00C77E407F0B7C017D187B041260C77E40DB
:10008E007F1C7C017D207B051260C77E407F177C24
:10009E00017D287B051260C77E407F217C017D306B
:1000AE007B051260C77E407F267C017D387B041263
:1000BE0060C77E407F2A7C017D407B041260C77E34
:1000CE00407F2E7C027DA07B091260C77E407F3769
:1000DE007C027DC07B071260C77E407F3E7C027D26
:1000EE00E07B051260C77E407F437C037D007B056D
:1000FE001260C77E407F487C037D207B051260C75F
:10010E007E407F4D7C037D407B051260C77E407F25
:10011E00527C037D607B091260C77E407F5B7C034F
:10012E007D807B091260C77E407F647C037DA07B4F
:10013E00091260C77E407F6D7C037DC07B1112600B
:10014E00C77E407F7E7C037DE07B071260C77E40CA
:10015E007F857C047D007B071260C77E407F8C7C90
:10016E00047D207B071260C77E407F937C047D4018
:10017E007B071260C77E407F9A7C047D607B0512F0
:10018E0060C77E407F9F7C047D807B051260C77EAA
:10019E00407FA47C047DA07B051260C77E407FA9B2
:1001AE007C047DC07B051260C77E407FAE7C047DE3
:1001BE00E07B051260C77E407FB37C057D007B052A
:1001CE001260C77E407FB87C057D407B091260C7F8
:1001DE009000297417F07F031263D69000287419CB
:1001EE00F090002074B1F09000217491F0900022F4
:1001FE007403F0900023747FF090002404F09000BC
:10020E00257403F0E4900026F0900027F090003063
:10021E0074091252697415F0A37403F0A3741512C5
:10022E0052697409F0A37403F0E4FFEFFD3395E017
:10023E00FC74302DF58274001252BB74102DF582B1
:10024E0074003CF583EEF00FBF08E0E4FFEFFD33E2
:10025E0095E0FC74382DF58274001252BB74182D83
:10026E00F58274003CF583EEF00FBF08E090052098
:10027E00E4F0A374B4F0900522E4F0A374B4F0900B
:10028E0005247401F0A374E0F0900526E4F0A37445
:10029E0078F09005287402F0A37458F090052AE4C3
:1002AE00F0A3743CF090052C7402F0A37458F07413
:1002BE000790052EF0A3F0900530F0A3F0900532D4
:1002CE00F0A3F0900534F0A3F0900536E4F0A3749B
:1002DE003CF0900538740AF09005397428F09005BA
:1002EE003A7405F090053B740AF090053CF09005C9
:1002FE003D7428F09000A47401F0900B607415F01A
:10030E00A37411F09000A57401F0900B807415F099
:10031E00A37410F09000A67401F0900BA07415F069
:10032E00A37421F09000A77401F0900BC07415F027
:10033E00A37420F09000A87401F0900BE07415F0F7
:10034E00A37431F09000A97401F0900C007415F0B4
:10035E00A37430F09000AA7401F0900C207415F084
:10036E00A37441F09000AB7401F0900C407415F042
:10037E00A37440F09000AC7401F0900C60745312B2
:10038E00525774361252577438F0A3E4F0A37453D4
:10039E00F0A3E4F09000AD04F0900C807453125270
:1003AE00577434F0A37421F0A37453F0A3E4F090C7
:1003BE0000AF04F0900CC01252557430F07403125A
:1003CE0052B3E4F09000B004F0900CE01252557469
:1003DE0030F074041252B3E4F09000B104F0900DBA
:1003EE000012524D74321252577452F0A37420F010
:1003FE009000B27401F0900D2012524D7432F0A3A1
:10040E0074021252B47420F09000B37401F0900D87
:10041E004074531252577433F0A3E4F09000B404B6
:10042E00F0900D6012527E7430F0740212525E9093
:10043E0000B57401F0900D8012527E7430F0740588
:10044E0012525E9000B67401F0900DA012527E749E
:10045E0030F0A3740612525F9000B77401F0900D45
:10046E00C012527E1252927498F0A3744B12525FC5
:10047E009000B87401F0900DE012527E12529274F8
:10048E0093F0A3741812525F9000B97401F0900E9D
:10049E000012527E7430F0A3741312525FA3747064
:1004AE00F0A37402F09000BA14F0900E201252874E
:1004BE007412F0A374701252577461F0A314F0907A
:1004CE0000BB7401F0900E4012528774111252A3A9
:1004DE009000BC04F07461900E6012528974141274
:1004EE0052A39000D104F090110012527E7492F03B
:1004FE00A3744BF0A37490F0A37402F0A37490F065
:10050E00A37432F07499A3F0A3F0A374601252573F
:10051E0074911252577491F0A3E412525F90000F2F
:10052E007401F0125DCE7F01126E9A7F401200169A
:10053E007D2F7F071266757D0C7F031266757D32E7
:0C054E007F061266757D1E7F0512667523
:01055A00227E
:0A60C7008E5A8F5B8C5C8D5D8B5E42
:1060D100E4F9C3E55E6480F8E96480985022E9FF41
:1060E1003395E0FEE55B2FF582E55A3EF583E493B7
:1060F100FDE55D2FF582E55C3EF583EDF00980D28B
:01610100227B
:10555B00AF6AEF3395E0FEE56975F008A42428F5F2
:10556B0082E43400F583E5822FF582E5833EF583F3
:10557B00E0FFE56AFD3395E0FC22AB66AD65AF64F9
:10558B00223EF583E0FD74B82FF582741D3EF58342
:10559B00EDF0056AE56A22EF3395E0FEEF25E0FFBB
:1055AB00EE33FE22A2E0CE13CE13223CF583EFF0B6
:0555BB00056AE56A220B
:045B7F008C5B8D5C52
:105B8300EF6043D201D202D20CE4F55D855C8285DD
:105B93005B83E0FEA3E04E6027AF5D1255A2E55C98
:105BA3002FF582E55B3EF583E0FEA3E0FF12471C81
:105BB300922820280B055DC3E55D6480949040CC5A
:065BC300C201C202C20C87
:015BC90022B9
:045BCA008C608D61FD
:105BCE00EF6043D201D202D20CE4F5628561828588
:105BDE006083E0FEA3E04E6027AF621255A2E5613E
:105BEE002FF582E5603EF583E0FEA3E0FF12471C31
:105BFE00922C202C0B0562C3E5626480949040CCFD
:065C0E00C201C202C20C3B
:015C1400226D
:04471C00AD07AC0633
:10472000C22D780CEF0880031255AFD8FB540FF55B
:10473000637808AF05AE04EF0880031255AFD8FBCD
:10474000540FF5647804AF05AE04EF0880031255EA
:10475000AFD8FB540FF565ED540FF566E563606463
:10476000B40108125585123BA88059E563B40208CC
:10477000125585126AC1804CE563B4030812558551
:104780001239CE803FE563B405081255851223C463
:104790008032E563B40608125585120A548025E577
:1047A00063B40708125585125AE88018E563B40807
:1047B0000812558512573A800BE563B40906125565
:0647C00085126874A22DB1
:0147C60022D0
:103BA8008F678D688B69E567B40113900020E0FF8B
:103BB8001258A3900020EFF0FD7F20023C65E567D6
:103BC800B40211900021123C6B900021EFF0FD7FB0
:103BD80021023C65E567B40311900022123C6B900A
:103BE8000022EFF0FD7F22023C65E567B4041090E7
:103BF8000023123C75900023EFF0FD7F23805EE5E3
:103C080067B40516900024123C75900024EFF0FD6F
:103C18007F247E0012636B0264CFE567B4061090C0
:103C28000025123C7F900025EFF0FD7F25802EE5D2
:103C380067B40710900026123C7F900026EFF0FD35
:103C48007F268019E567B40819900027E0FFAB6963
:103C5800AD681258A3900027EFF0FD7F277E001271
:103C6800636B22E0FFAB69AD681258A322E0FFAB9B
:103C780069AD681258A322E0FFAB69AD681258A37A
:013C88002219
:1058A300D22EAC07BD01047E018033BD02047E020B
:1058B300802CBD03047E048025BD04047E08801E65
:1058C300BD05047E108017BD06047E208010BD0731
:1058D300047E408009BD08047E808002C22EBB0185
:1058E30005EE4204800BEB7006EEF452048002C214
:0758F3002E302E03AF04224A
:0158FA00228B
:026AC1008B67E1
:106AC300C22EEF7016ED7013E5677003025C60E58C
:0B6AD30067B401077880E6FF125A4C00
:016ADE002295
:0639CE008F678D688B6914
:1039D400E5677007123AB4E4FD801AE567B401079D
:1039E400123AB47D01800EE567B4020CAD69AF688C
:1039F400126E377D02024EC2E567B40306124F4AC7
:103A0400C21D22E567B40415AD69AF6812640A8F5C
:103A140043754205E5427003023AB380F7E56764F3
:103A2400067017E5687013F56A12555B74102DF56E
:103A34008274001255B6B408F022E5676407701763
:103A4400E5687013F56A12555B74182DF5827400DD
:103A54001255B6B408F022E56764087027E568706B
:103A640023E569701FF56AAF6AEF3395E0FE7410C1
:103A74002FF582740012558CB408EC754201E542AE
:103A8400602D80FAE56764097025E5687021E569B1
:103A9400701DF56AAF6AEF3395E0FE74182FF58256
:0F3AA400740012558CB408EC754201E54270FCB9
:093AB30022AD69AF68126E3722E2
:1023C4008F678D688B69E5677018E5687014E56937
:1023D40070057F01126E53E5696401600302257183
:1023E4008043E567701CE568B40117E56970057FF3
:1023F40004126E53E569640160030225717F0402CF
:10240400256EE5677029E56864027023E569700547
:102414007F05126E53E56964016003022571900023
:102424000FE0B403057F0102256E7F0502256EE5EA
:1024340067B4011BE5687017E56970057F02126EC9
:1024440053E569640160030225717F0202256EE58C
:1024540067B4011CE568B40117E56970057F0812CB
:102464006E53E569640160030225717F0802256EDD
:10247400E56764017029E56864027023E569700505
:102484007F0A126E53E569640160030225719000AE
:102494000FE0B403057F0202256E7F0A02256EE574
:1024A40067B4021BE5687017E56970057F40126E1A
:1024B40053E569640160030225717F4002256EE5DE
:1024C40067B4021CE568B40117E56970057F101252
:1024D4006E53E569640160030225717F1002256E65
:1024E400E56764027024E5686402701EE56970059E
:1024F4007F50126E53E5696401707290000FE0B46E
:1025040003047F4080647F508060E567B40317E56F
:10251400687013E56970057F80126E53E569640184
:10252400704B7F808044E567B40318E568B40113F9
:10253400E56970057F20126E53E5696401702E7F92
:10254400208027E56764037024E5686402701EE553
:102554006970057FA0126E53E569B4011090000FF5
:0E256400E0B403047F8080027FA012001622E4
:060A54008F678D688B69BD
:100A5A00C22EE5677019AD69AF68126E378E348F92
:100A6A0035D3E5359400E534940050F5020D12E5CE
:100A7A0067B4011BE568B40116E5697007C22F7FE8
:100A8A0001122F1AE56964016003020D128058E50C
:100A9A00676401702BE56864027025E5697007C216
:100AAA002F7F02122F1AE56964016003020D12906A
:100ABA00000FE064037003020D12D22F7F0280310F
:100ACA00E56764017031E5686403702BE5697007B6
:100ADA00C22F7F03122F1AE56964016003020D1207
:100AEA0090000FE0B40306D22F7F018004D22F7F3B
:100AFA0003122F1A020D12E5676401702DE568646E
:100B0A00047027E569700CC22F7F01122F1A7F40EB
:100B1A00126E53E56964016003020D12D22F7F0140
:100B2A00122F1A7F40120016807CE5676401703A22
:100B3A00E56864057034E569700CC22F7F02122FD4
:100B4A001A7F10126E53E56964016003020D129058
:100B5A00000FE064037003020D12D22F7F02122FDE
:100B6A001A7F10120016D22F803EE5676401703E8C
:100B7A00E56864067038E569700CC22F7F03122F8E
:100B8A001A7F50126E53E56964016003020D12D296
:100B9A002F7F03122F1A90000FE0B403047F4080C6
:100BAA00027F50120016C22F12692B020D12E5673E
:100BBA0064027031E5686401702BE569700A7F1080
:100BCA00120D2254FE020D01E569B4010A7F1012CA
:100BDA000D2A4401020D01E56964026003020D1247
:100BEA007F01020D0DE56764027031E568640270E9
:100BFA002BE569700A7F20120D2254FD020D01E5D2
:100C0A0069B4010A7F20120D2A4402020D01E56926
:100C1A0064026003020D127F02020D0DE567640291
:100C2A007031E5686403702BE569700A7F40120D24
:100C3A003254FB020D01E569B4010A7F40120D3AF4
:100C4A004404020D01E56964026003020D127F0388
:100C5A00020D0DE5676402702FE56864047029E5EA
:100C6A0069700A7F80120D3254F7020D01E569B4EA
:100C7A0001097F80120D3A4408807CE569640260AC
:100C8A0003020D127F04807BE56764027033E56816
:100C9A006405702DE569700D7F04126E879000243B
:100CAA00E054EF8052E569B4010D7F04126E9A9008
:100CBA000024E044108040E5696402704B7F05809F
:100CCA0042E56764027041E5686406703B7D017F16
:100CDA0007124E3A4032E569700D7F08126E87900E
:100CEA000024E054DF8010E569B401107F08126E19
:100CFA009A900024E04420F0D22E800CE569B402D8
:100D0A00077F06123054C22E302E0C900024E0FDCC
:070D1A007F247E0012636BD1
:100D210022126E87900024E022126E9A900024E035
:100D310022126E87900024E022126E9A900024E025
:010D4100228F
:025AE8008B67CA
:105AEA00EF7037ED7034E567700690000F04802080
:105AFA00E567B4010A90000F7402F0D22E801BE50C
:105B0A0067B40216C21D7FFF126E5390000F740312
:105B1A00F0C22F7F02122F1AD22E302E0C90000FB5
:095B2A00E0FD7F0F7E0012636BA9
:015B3300224F
:10573A008F678D688B69E567700C12577E749F2F8F
:10574A00F58274008019E567B4010C12577E749FC4
:10575A002FF58274008016E567B402091257863E57
:10576A00F583E4F022E567B403091257863EF58310
:10577A007401F022AD69AF68126E3722AD69AF6865
:0B578A00126E37746F2FF5827400223E
:026874008F672C
:10687600AF057804EF08800123D8FD4BF568E5677E
:10688600B40908E568B499030253B0AD68AF67125E
:0268960064FF9D
:0168980022DD
:0D6E3700EF75F00AA47C002DFFEC35F0FE95
:016E4400222B
:0D6E4500C296007F0512679212643CD2963F
:016E5200221D
:106CC600126E45EF20E0F9C296007F06126792C267
:066CD600B60000D2962278
:106CDC00126E45EF20E0F9C296007F04126792C253
:066CEC00B60000D2962262
:045F97008E608F6128
:105F9B00AE04AF058E638F64C296007F03126792C7
:105FAB00E560FF126792AF61126792E4F5621264CB
:105FBB003CE5642562F582E43563F583EFF0056219
:095FCB00E562C3942040E7D29680
:015FD40022AA
:085C15008E658F668C678D68B7
:105C1D00126E45EF20E0F985656A85666BC29600C8
:105C2D007F02126792E567FF126792AF6812679263
:105C3D00E4F569E56B2569F582E4356AF583E0FFE6
:105C4D001267920569E569C3942040E7C2B600006A
:025C5D00D296DD
:015C5F002222
:0A54F5008E5A8F5B8C5C8D5D8B5E20
:1054FF00C2AF126CC6126E45EF20E0F9855C608575
:10550F005D61C296007F02126792E55AFF126792A1
:10551F00AF5B126792E4F55FAF5EEF3395E0FEC3CA
:10552F00E55F9FEE6480F87480985014E561255F05
:10553F00F582E43560F583E0FF126792055F80D84E
:0B554F00C2B60000D296126CDCD2AF96
:01555A00222E
:10636B008E718F728D73C2AF126CC6126E45EF2099
:10637B00E0F9C296007F02126792E571FF126792F5
:10638B00AF72126792AF73126792C2B60000D296C9
:06639B00126CDCD2AF22FF
:10604F00C2AFE4F55BF55CF55DF55EF55FF55AAE55
:10605F005EAF5FAC5BAD5C125F977420255CF55C47
:10606F00E4355BF55B7420255FF55FE4355EF55E27
:0B607F00055AE55AC3948940D6D2AF01
:01608A0022F3
:105DCE00C2AF756200756300756400E4F560F5613D
:105DDE00F55F126CC6AE63AF64AC60AD61125C155C
:105DEE0074202561F561E43560F56074202564F555
:105DFE0064E43563F563055FE55FC3948940D312B0
:045E0E006CDCD2AFC7
:015E1200226D
:105622000500050105030507050F051F051E051CDD
:10563200051805100201040E040A03060101040BF9
:105642000304040F020304010302040D0200020218
:10565200030004090404030503070100030304070C
:10566200030104060402040C0516051500000615C4
:0E567200062A060C06380633061E0612061718
:104C93002430F58274003EF583EDFF3395E0FEE5A5
:104CA300822FF582E5833EF583E0FFEDFB3395E04C
:104CB300FA22AF41126792C293126E91D293D2AF8E
:104CC300223EF583E0FC74B82FF582741D3EF58314
:104CD300ECF00D221528E528D394002225E02422A8
:104CE300F582E43456F583E49322E4F57CD20EC2D4
:104CF30026C21CC219227FA0126E53E4F542C21DC4
:104D030022126E91D2B67801EF0822122B57D2CA23
:0F4D1300D20ED22622ECFF3395E0FEEF7803227A
:1040C100200E2F900540E004F577D3648094815051
:1040D10003024181D3E5776480948F400375770FA4
:1040E100900029E0FF122B5790002AE0F576124C40
:1040F100ED22301958302612124CD740030241816B
:10410100C2CAC226D21C85762822301C0A124CD77C
:10411100506EC226C21C22AF7A157AEF700BC219FB
:10412100E57625E0F528D21C22E57B30E005857691
:10413100288008E57675F003A4F528AF7B7801EFB8
:1041410008800103D8FDF57BD226D2CA22D5770893
:10415100C20EE4F542C21D22057C7440257CF58225
:10416100E43405F583E0124CDF540FF57A740193C2
:10417100F57B700AD21CE57625E025E0F528D219F9
:01418100221B
:1050DB00200E12900029E0FF122B5790002AE0F5CA
:1050EB0078124CED2230195130260F124CD7505DEF
:1050FB00C2CAC226D21C85782822301C0A124CD771
:10510B00504BC226C21C22AF7A157AEF7007C21918
:10511B00C20EF54222E57B30E0058578288008E554
:10512B007875F003A4F528AF7B7801EF08800103B5
:10513B00D8FDF57BD226D2CA22E543124CDFFA7496
:0D514B000193FBEA540FF57AEBF57BD219C6
:015158002234
:10643C00E4F575D297F574C2B6126E91AF7578010A
:10644C00EF08800123D8FDF57530970343750112D1
:10645C006E91D2B60574C3E5746480948840D8AF4D
:01646C0075BA
:01646D00220C
:096E9100000000000000000022D6
:10664900C2B7E4FEC2B6126E91EF30E704D2B5804C
:1066590002C2B5124D04800123D8FDFF126E910EBE
:0B666900BE08E1C2B6D2B7D2B6D2B56F
:016674002203
:0D001600C2AFEF4227AF27126649D2AF22DA
:0E6E5300C2AFEFF45227AF27126649D2AF222A
:10679200E4FEC2B6126E91EF30E704D2B58002C2B7
:1067A200B5124D04800123D8FDFF126E910EBE0872
:0567B200E1D2B6D2B5F2
:0167B70022BF
:096E9A00C2AFEF4241124CB522D7
:0A6E8700C2AFEFF45241124CB522E5
:102B5700EF123B822BBF012BC6022BCD032BD404D4
:102B67002BDB052BE2062BE9072BF0082BF7092BAC
:102B7700FE0A2C050B2C0C0C2C130D2C1A0E2C21D9
:102B87000F2C28102C2F112C36122C3D132C4414EB
:102B97002C4B152C52162C59172C60182C67192CF6
:102BA7006E1A2C751B2C7C1C2C7E1D2C851E2C8CC8
:102BB7001F2C932000002C7C75CB8E75CAC62275FE
:102BC700CB9575CA772275CB9B75CA692275CBA041
:102BD70075CABA2275CBA675CA332275CBAB75CA2F
:102BE700632275CBB075CA022275CBB475CAA3220E
:102BF70075CBB875CAFA2275CBBC75CAD82275CB06
:102C0700C075CAA82275CBC475CA362275CBC775DD
:102C1700CA862275CBCA75CABC2275CBCD75CAB414
:102C27002275CBD075CA762275CBD375CA3022757B
:102C3700CBD575CAB22275CBD875CA132275CBDA34
:102C470075CA522275CBDC75CA7D2275CBDD75CA74
:102C57006E2275CBE075CA542275CBE275CA1B226A
:102C670075CBE375CAC32275CBE575CA5E2275CBF2
:102C7700E675CADA22801C75CBE875CA902275CB37
:102C8700EA75CAD92275CBEC75CA092275CBED75E1
:0A2C9700CA292275CBE875CA412254
:10002600C3EF648094A15008EF25E025E0F528226F
:04003600E4F52822A3
:023602008F5ADD
:10360400900118E0FFE55A7006E545D39F5012E596
:103614005A640160030236F8E546D39F500302362C
:10362400F8E55A7018C3E5459FF55D74602FF5827F
:10363400E4341EAD82F55E8D5F7F40801BE55AB495
:103644000119C3E5469FF55D74B02FF582E4341E7D
:10365400AF82F55E8F5F7F101200167FF47E011239
:103664006BC97D207F051266757D1A7F0812667509
:103674007FC87E00126BC9E4F55BE55BC3955D50C2
:1036840061055FE55FAE5E7002055E14F5828E83B0
:10369400E0F55C123B8236D50036B30A36B70B36FA
:1036A400BD0C36C30D36C90E36CF0F000036DBE431
:1036B400FD80277D5F7F0780227D5E7F06801C7DE5
:1036C4000A7F0280167D327F0280107D467F028051
:1036D4000A7D0A7F038004AD5CE4FF126675055B16
:1036E4008098E55A70047F408007E55AB401057F4D
:0436F40010126E53EF
:0136F80022AF
:10505800200E10754406901DB8E06003D20E22E4BD
:10506800F54222E528D394004003152822C2CA1528
:1050780044E54414603D14603214601D1460151436
:105088007049901DB8E0FF7003F54222122B57902B
:105098001DB9802F901DBA8015901DBBE0FF7003CD
:1050A800F54222122B57901DBC8018901DBDE0FFC1
:1050B800020026901DBEE0FF7003F54222122B5716
:1050C800901DBFE0FF120026D2CA22E4F542C2CAF0
:0350D800C20E22E3
:1065ED00900028E0FF6026200E07124D0E7528142E
:1065FD0022E528D394004003152822202608D2CA6C
:0E660D00752814D22622C2CA75287DC2262204
:10658F00200E0C7F1C124D0E75286475793C22E588
:10659F0028D394004003152822AF791579D3EF64DF
:0E65AF00809480400475286422C20EE4F542F8
:0165BD0022BB
:10629200E54214601C14601C14601F146022146018
:1062A2002224057021C2CAC20EC226C21CE4F544D1
:1062B200220250581265EDD21D221240C1D21D2277
:0762C20002658F1250DB2280
:1063D600BF010790002A7418F022BF020790002A16
:1063E6007412F022BF030590002A8014BF040790A0
:1063F600002A740BF02290002ABF05047409F022CB
:04640600740CF02200
:024FD200AC072A
:104FD400C3EC64809480404AEC64809488504320FD
:104FE4002A21E4FD124D18C333CE33CED8F9124C26
:104FF4009374102BF58274003AF583EFF00DBD081D
:10500400E3801FE4FD124D18C333CE33CED8F9121A
:105014004C9374182BF58274003AF583EFF00DBDB0
:1050240008E3202A16E4FDEDFF3395E0FE74102F0B
:10503400F5827400124CC4BD08ED22302A15E4FD3B
:10504400EDFF3395E0FE74182FF5827400124CC402
:03505400BD08EDA7
:015057002236
:1053B0007D3F7F091266757D507F08126675906E7D
:1053C000C31254177D5B7F06126675906EC412542B
:1053D00017906EC5E493FDE4FF126675906EC6E407
:1053E0009324BE601414601514601814601B1460BC
:1053F0001E240570217D0A80067D3280027D467F55
:105400000280107D0A7F03800A7D287F0380047D4F
:10541000467F0312667522E493FDE4FF126675224F
:105ED9008F5BE55B7005D22CFF8009E55BB4010798
:105EE900D22C7F011259A97D4B7F021266757D0262
:105EF900E4FF1266757D32E4FF1266751253B0E550
:105F09005B70028005E55BB401057F40126E532288
:103C8900A209300501B350307D017F04124E3A502C
:103C99002320050E30090B9000A4E0FF7C0B7D600A
:103CA900800F30050F20090C9000A5E0FF7C0B7DEB
:103CB90080125BCAA2099205A20A300601B35030EC
:103CC9007D027F04124E3A502320060E300A0B90D3
:103CD90000A6E0FF7C0B7DA0800F30060F200A0CA8
:103CE9009000A7E0FF7C0B7DC0125BCAA20A920676
:103CF900A20B300701B350307D037F04124E3A50B6
:103D09002320070E300B0B9000A8E0FF7C0B7DE011
:103D1900800F30070F200B0C9000A9E0FF7C0C7D71
:103D290000125BCAA20B9207A20D300801B35030F2
:103D39007D047F04124E3A502320080E300D0B905B
:103D490000AAE0FF7C0C7D20800F30080F200D0CAD
:103D59009000ABE0FF7C0C7D40125BCAA20D92087B
:013D69002237
:1064CF00534103900024E0FE543FFF7804088001FD
:1064DF0023D8FD54F0FFEE30E4034307049000246B
:0F64EF00E030E503430708EF4241C2AF124CB55E
:0164FE00227B
:023054008F6A81
:10305600E56A64017023AF417803EF08800123D845
:10306600FD33922F7F10202F081231407F1002313E
:103076003412314B7F1002313CE56A64027023AF93
:10308600417802EF08800123D8FD33922F7F20205C
:103096002F081231407F2002313412314B7F20023B
:1030A600313CE56A64037023AF417801EF08800183
:1030B60023D8FD33922F7F40202F081231567F40B0
:1030C6000231341231617F4002313CE56A6404709A
:1030D60018E54133922F7F80202F071231567F80CB
:1030E600804C1231617F80804DE56A64057021AFA6
:1030F600417805EF08800123D8FD33922F7F042005
:103106002F0712316C7F0480251231777F048026C9
:10311600E56A64067023AF417804EF08800123D87E
:10312600FD33922F7F08202F0812316C7F08026E24
:09313600871231777F08126E9AAE
:10313F0022126E9A7FF47E01126BC922126E877F64
:10314F00F47E01126BC922126E9A7FF47E01126B0C
:10315F00C922126E877FF47E01126BC922126E9AFA
:10316F007FF47E01126BC922126E877FF47E0112EB
:03317F006BC922F7
:105D3D00900024E030E0057F10126E9A900024E070
:105D4D0030E1057F20126E9A900024E030E2057F4D
:105D5D0040126E9A900024E030E3057F80126E9A17
:105D6D00900024E030E4057F04126E9A900024E048
:095D7D0030E5057F08126E9A2240
:106C1A0030030A124CF9C203C210C21D2230040901
:0A6C2A00124CF9C204C212C21D226E
:1064FF008F708D71E570B4011FE5717003125C60D0
:10650F00E571B401077880E6FF125A4CE571B43299
:10651F000E7FF47E01026BC9AD71AF7012667522EA
:10667500EFFEEDFF1280008E2D8F2E12533B7574A9
:1066850032AF741574EFD39400400EE4F573E573DF
:09669500C3943A50EC057380F542
:01669E0022D9
:10533B00D2A8AFA875A881C213852E82852D83E4D0
:10534B0093C4540FFE4306F08E80C284D28500C2F4
:10535B00870000D287007580FF7580FEC284C285EE
:10536B0000C2870000D287007580FFD2137D407C7E
:10537B001FE4FE30B40D0EBE32F9ED1D70011CEDB5
:10538B004C70EE7C1F7D40E4FE20B40D0EBE32F956
:10539B00ED1D70011CED4C70EE8FA8C2A87F0A7E2C
:0453AB0000126BC9B8
:0153AF0022DB
:10669F007580FDC284C28500C28700000000D287CA
:1066AF00007580FF7F0A7E00126BC97F997E0912E9
:0A66BF0080008E2D8F2E12533B2217
:10418200D284D285C286A2809216A281921FA28276
:104192009217A2839220D2862001537D027F0112C0
:1041A2004E3A40137D037F01124E3A400A30160701
:1041B200301832D22380377D027F01124E3A500FDF
:1041C20030160C301F09301804D223802180167D4E
:1041D200037F01124E3A5012201603301F0C301882
:1041E20004D22380091267B88004C218C2232002B5
:1041F2004E7D027F02124E3A40127D037F02124E22
:104202003A4009301706301A2FD224227D027F024B
:10421200124E3A500E30170B302008301A03D224B7
:104222002280157D037F02124E3A500F2017033071
:104232002009301A03D224220267DEC21AC22422C3
:1067B800753D1E753E60E4FFE53E2FF582E4353DEC
:1067C800F583E4F00FBF50F0753D1E753E60E4F5AB
:0567D80045C225D218A6
:0167DD002299
:1067DE00753F1E7540B0E4FFE5402FF582E4353F6E
:1067EE00F583E4F00FBF10F0753F1E7540B0E4F571
:0567FE0046C227D21A7B
:016803002272
:106B7300C284D285C286A2809209A281920AA2828D
:0D6B8300920BA283920DD286D284D285227D
:10610200E57E2560F582E4357DF5832274FF123B3E
:1061120058E4FBFAF9F8C3023B45057F7480257EFB
:10612200F57EE4357DF57D22F582E4341DF583228A
:0B613200757F01757D00757E20E42262
:104242007D027F07124E3A50057F04126E87C22804
:10425200D222E4F5427FE87E03126BC9C298C2AF54
:10426200C22F7F03122F1A755E7F755D96755C985B
:10427200755B00785B12610E504430983E12000666
:10428200126DAAEF14601824F0602624C1600B247A
:10429200F670287F06126EAC80211261B2801C7FFC
:1042A20006126EAC1269711264CF125DCED22880F2
:1042B2000A7F06126EAC1259FCD2283028B5E47877
:1042C20085F6D22F7F01122F1A7F40120016C22FBD
:1042D20012692B7D467F021266757D1E7F0712666C
:1042E200757D147F081266757D327F03126675C272
:0D42F2002F7F03122F1A7FFF126E53C2227E
:0142FF00229C
:1059FC00126132F55F7F02126EACE57F2402F56115
:105A0C00AF7F126EACE4F560126102E0FF126EAC77
:105A1C00126102E02561F5610560E560C394804088
:105A2C00E7AF61126EAC7F03126EAC126EB4EF6412
:0F5A3C0015600C12611C055FE55FC3942240B634
:015A4B002238
:10697100126132F55F1266C950077F06126EAC8054
:10698100057F15026EAC12611C055FE55FC39422A1
:0269910040E3E1
:0169930022E1
:1066C900E4F560126EB474D0256012612AEFF0050A
:1066D90060E560C3948440EB126D88901E52E0B56A
:0866E9000705126BE4D322C384
:0166F1002286
:106BE400E4FF74D22FF582E4341DF583E0FEE57EE4
:0A6BF4002F126106EEF00FBF7FE8DC
:016BFE002274
:106D8800E4FFFE74D02E12612AE02FFF0EBE82F3BC
:016D980022D8
:1061B200E4F55FF5657564E0756393756204F561F6
:1061C200786112610E50213098F61200068F60E558
:1061D2006064046013AF65056574D02F12612AE50F
:0861E20060F0255FF55F80D835
:0161EA002292
:04000600AF99C29854
:01000A0022D3
:086EAC003099FDC2998F992273
:076EB4003098FDAF99C29870
:016EBB0022B4
:106C80000C0102030405060708090A0B0C010203A4
:086C90000405060708090A0BC0
:1066F200AF5FEF3395E0FE75F007EF123B76EE7574
:10670200F007A42583F583E0227883E6FF126C4E1E
:09671200EF22C295D297D2AF220A
:10680400C22BC2AF126EBC7F83126C98126A8212C2
:1068140067147884E66F600B125E56302A05125FA7
:0568240019922BA22BCC
:01682900224C
:105F19007984E778876660367884E6FF7887F6EFD4
:105F29007013E552C3940A500C7D077F04124E3A50
:105F39005003125E137D057F04124E3A5010E5415D
:105F490054036005123F24D322123F24C322C322E3
:103F2400E4F55F900A501266F27003023FE8900ACB
:103F3400511266F960167881666003023FE8900AC0
:103F4400521266F27888666003023FE8AF5FEF338F
:103F540095E0FE900A531266F9FF7880E6FEEF6E54
:103F64006020EF601DB4080BEED394014005EE947D
:103F740007400FEF6409706CEE64016005EE64079E
:103F84007062AF5FEF3395E0FE900A541266F9FF5A
:103F9400F46006EF788366704BE55FFD3395E0FCD3
:103FA400900A5575F007ED123B76EC1267017884A0
:103FB400667031D201D20274BD2DF58274003CF5D5
:103FC40083E0FFC007EDAE047805C333CE33CED80B
:103FD400F92480F582740E3EAD82FCD007125BCAD0
:103FE400C201C202055FC3E55F648094935003027B
:023FF4003F2765
:013FF60022A8
:105E13007D087F04124E3A500D7883E6FF126C4ED4
:105E2300EFC39407402CD22F7F01122F1A7F401209
:105E33000016C22F12692BD201D202E4FD7F0A128F
:105E43004EC2C201C2027F50126E53C22F7F011293
:035E53002F1A22E1
:105E5600C2AF126EBC7FBF126C98126A827884A69B
:105E660007126A827884A607126A827883A60712C6
:105E76006A827888A607126A827881A607126A82E1
:105E86007880A607126A827882A607126EBC12670D
:025E96001422D4
:10579500C2AF126EBC7F8E1257E47F90126C987F59
:1057A500A7126C98126EBC7FBE126C98E4FF126C47
:1057B500987884E6FF126C987883E6FF126C9878E7
:1057C50088E6FF126C987881E6FF126C987880E67F
:1057D500FF126C987882E6FF1257E41267142212C2
:0B57E5006C98E4FF126C98126EBC225E
:105A4C008F72E572B401047D63803EE572B4020688
:105A5C007D087F068035E572B403067D317F0880B2
:105A6C002AE572B404067D617F08801FE572B405D7
:105A7C00067D257F088014E572B406067D597F03E8
:0F5A8C008009E572B407077D487F07126675220F
:026C4E00AE078F
:106C5000EE54F0FF780408800103D8FD75F00AA413
:066C6000FFEE540F2FFFB0
:016C6600220B
:105C600012670B906C8093FF123503788412670DD6
:105C7000601B788412670DC3940A50077D327F063B
:105C80001266757884E6FF126C4E12350312670BAC
:105C9000C3940C50067D0A7F0280047D507F06125B
:0A5CA00066757D507F0512667522BF
:105953007FF47E01126BC97D097F0612667578811B
:105963001259997D0E7F031266757D357F06126687
:10597300757D097F0612667578881259997D1E7F99
:10598300091266757D1E7F071266757882E6FF121F
:105993006C4E12350322E6FF126C4E1235037FF470
:0659A3007E01126BC92217
:076EBC00C2B6C295D2952277
:106C9800E4FEC297EF30E002D297C2B6D2B6EFC395
:066CA80013FF0EBE08EC14
:016CAE0022C3
:106A8200E4FFD297FED2B6C2B6A297E433C4333340
:0F6A9200335480FDEFC313FFED42070EBE08E63D
:016AA10022D2
:1056DD00EF3395E0FE74702FF58274003EF583E094
:1056ED00FF22AF5AEF3395E0FEEF222460F582746E
:1056FD00013EAD82FCD22822900520E0F547A3E0C3
:10570D00F548222450F58274053EAD82FC229000AE
:10571D00BAE0FF7C0E7D2022D221D201E4FF22C20D
:0D572D0001C2217F1922D221D22F7F02223A
:1028A200E5527008126C678F5202299DE552B405F9
:1028B200081245198F5202299DE552B40B08126C79
:1028C200F28F5202299DE552B40A08125CAA8F5275
:1028D20002299DE552B40F081260128F5202299DFF
:1028E200E552B414081225728F5202299DE552B4A2
:1028F2001908126ADF8F5202299DE552B41E08128E
:1029020069DA8F5202299DE552B42308126A408F78
:102912005202299DE552B42807126E618F52807BC4
:10292200E552B42D0712676B8F52806FE552B432B5
:10293200071261EB8F528063E552B43E07126AFDC3
:102942008F528057E552B43C07126D528F52804B22
:10295200E552B43307126A1E8F52803FE552B441EA
:1029620007126DDB8F528033E552B44C07126DEBC8
:102972008F528027E552B44407126DFB8F52801BA1
:10298200E552B4370712584A8F52800FE552B439D4
:10299200071257F08F528003E4F552E55370061286
:1029A200000E8F5322E553B40506126EA38F5322F5
:1029B200E553B40A06126E0B8F5322E553B40F0689
:1029C200126E1A8F5322E553B41406123E4A8F53E5
:1029D20022E553B43D06126B1B8F5322E553B43FDD
:1029E2000612652F8F5322E553B443061267438FB5
:1029F2005322E553B44D06126A618F5322E4F55314
:012A020022B1
:106C67007D077F05124E3A500D30000A90052AE045
:096C7700F52BA3E0F52C7F0522AA
:10451900302314200F11C21B7D047F01124E3A5023
:10452900037F0B227F0A227F081262C950061243B9
:10453900B67F0022202308300F05C20F7F05227D98
:10454900057F06124E3A501EE5394538701890001D
:10455900B5E0FF7C0D7D80125BCA90052EE0F53831
:10456900A3E0F53980487D067F06124E3A501EE5D4
:104579003C453B70189000B6E0FF7C0D7DA0125BB6
:10458900CA900530E0F53BA3E0F53C80217D077F2B
:1045990005124E3A500D30000AE52C452B7004C225
:1045A90000800B7885E6B405057F04125159E55161
:0D45B900700875510AD22A1268047F05228D
:106CF20090053BE0F54E2023037F0522E54ED39419
:066D02000050F37F0A229D
:105CAA007D077F05124E3A500C7D077F05124E3A4A
:105CBA00503230002F7D017F01124E3A5026D22FEA
:105CCA007F01122F1A7F011200167D027F07124EE2
:105CDA003A50057F04126E9A9000A0E0FF7C0A7D7C
:0A5CEA00E0125BCA1257057F0F227B
:10601200302337E5484547700C7D087F01124E3A20
:1060220050037F372230030EE53A700A126C1A7F52
:106032000112001680113025037F14227885E6B400
:0D60420005057F031251597F0F227F1422A4
:1025720090053DE0F54B7F01126E53126C1A7D02FD
:102582007F07124E3A5009E54B70057F04126E87A1
:102592009000A1E0FF7C0B7D00125BCAD22A126878
:1025A20004E54570030226937C017D001227115039
:1025B200037F3E227C017D501226F150037F3C2294
:1025C2007C017D581226F150037F3C227C017D1054
:1025D2001226F9500812270150037F33227C017D15
:1025E200201226F9500B9000BBE0FF7C0E7D40804C
:1025F200207C017D28122709500512571B80127C6E
:10260200017D3012270950129000B9E0FF7C0E7D47
:1026120000125BCA1267B87F00227C017D40D2287B
:10262200E4FF1247C750037F4C227C017D381227FA
:102632001150037F44227C017D18C228E4FF124717
:10264200C7500C7D057F01124E3A50037F4122E4B0
:10265200F55A1256EF7803C333CE33CED8F9125659
:10266200F8E4FF1247C7501BAF5A1256DDC00712DB
:1026720056EF7805C333CE33CED8F9125710D007B0
:10268200125B7F055AC3E55A648094A840C47F193F
:1026920022122701500C7D077F05124E3A5041301D
:1026A200003E7885E670047F0180087885E6B404F0
:1026B200077F0212515980257D037F06124E3A5040
:1026C2001CE557455670169000AFE0FF7C0C7DC0AC
:1026D200125BCA900532E0F556A3E0F5577F192246
:0E26E2007D077F05124E3A50052000027F054D
:1026F00022D228E4FF1247C722D228E4FF1247C79C
:10270000227D077F05124E3A22D228E4FF1247C7E6
:0927100022C228E4FF1247C7228F
:106ADF003025031267B87D077F05124E3A50062006
:0E6AEF0000037F0522900538E0F54E7F1E2241
:1069DA00E54E70037F23227D027F07124E3A50094B
:1069EA00E54B70057F04126E873023037F0A227FEE
:0269FA001E225B
:106A40001257057D067F01124E3A500C9000ACE0C3
:106A5000FF7C0C7D60125BCA900539E0F54E7F2DFE
:016A60002213
:0E6E61007FA0126E53900539E0F54E7F2D2272
:10676B00D22A1268047D027F07124E3A5009E54B7C
:10677B0070057F04126E87E54E70037F3222302343
:07678B00037F0A227F2D228B
:1061EB00301D037F32227D047F06124E3A501FE58D
:1061FB0055455470199000B0E0FF7C0C7DE0125BAC
:10620B00CA900534E0F554A3E0F5557F3222C22F36
:08621B007F01122F1A7F0022FF
:106D520020210CD221E4FF12055BC2217F00227F99
:026D62003C22D1
:106AFD00202118D2217F40120016D201121E0BC286
:0E6B0D00017F40126E53C2217F19227F3E226B
:106DDB0020210A12572512360212572C227F4122EC
:106DEB0020210A12572512608B12572C227F442226
:106DFB0020210A12572512548C12572C227F442221
:05000E0000007F052247
:096EA3003024037F0A227F05223E
:0F6E0B009000A2E0FF7C0B7D20125BCA7F0F225C
:0F6E1A003024093027037F14227F0F227F142298
:103E4A009000A3E0FF7C0B7D40125BCAE54670033D
:103E5A00023F197D017F03124E3A50677C017D08AB
:103E6A00C2287F011247C750037F3F227C017D5041
:103E7A00123F1C50037F3D227C017D58123F1C508B
:103E8A00037F3D227C017D40D2287F011247C75023
:103E9A00037F4D227C017D28D2287F011247C7501B
:103EAA000912571B125BCA7F00227C017D18C228A7
:103EBA007F011247C7500C7D057F02124E3A50030C
:103ECA007F43227D027F03124E3A5043E4F55AAFF4
:103EDA005A1256F17803C333CE33CED8F91256F8B4
:103EEA007F011247C7501DAF5A1256DDC007AF5A9D
:103EFA001256F17805C333CE33CED8F9125710D003
:103F0A0007125B7F055AC3E55A648094A840C07FB4
:013F1A0000A6
:093F1B0022D2287F011247C722BF
:106B1B00202118D221C22F7F01122F1A7F01126E52
:0E6B2B00537F0112055BC2217F00227F3D22B5
:10652F0020212A125733122F1A7FF47E01126BC9C2
:10653F007F10120016D202121C0AC2027F10126EB6
:10654F0053C22F7F02122F1AC2217F00227F3F22B8
:10674300202122125733122F1A7FF47E01126BC9B4
:10675300D2027F01123602C202C22F7F02122F1A07
:08676300C2217F00227F4322C6
:106A610020211B125733122F1AD2027F0112608B81
:106A7100C202C22F7F02122F1AC2217F00227F4D34
:016A810022F2
:1055C000AF5AEF3395E0FE22900520E0F547A3E0C7
:1055D000F548222460F58274013EAD82FCD2282277
:1055E00074702FF58274003EF583E0FF22C202C280
:1055F000217F1922900522E0F549A3E0F54A2224F3
:1056000050F58274053EAD82FC22055AC3E55A640A
:105610008094A822D221C22F7F0122D221C22F7FC3
:02562000022264
:1032AF00E552700612661B8F5222E552B4050612C4
:1032BF0038DF8F5222E552B40B061269FC8F52226F
:1032CF00E552B40A0612446B8F5222E552B40F0630
:1032DF00126D648F5222E552B411061258FB8F52B1
:1032EF0022E552B412061251D38F5222E552B41472
:1032FF000612102D8F5222E552B419061265BE8F99
:10330F005222E552B41E0612655F8F5222E552B467
:10331F002306125E988F5222E552B42806126E6F62
:10332F008F5222E552B42D0612613D8F5222E55283
:10333F00B432061262238F5222E552B43C06126D4C
:10334F00768F5222E552B43D06126BFF8F5222E563
:10335F0052B43E061268998F5222E552B43F0612BC
:10336F006D998F5222E552B44106126AA28F5222F2
:10337F00E552B443061269948F5222E552B44C06BB
:10338F00126C348F5222E552B44D061269B78F5228
:10339F0022E552B4370612584A8F5222E552B439F9
:1033AF00061257F08F5222E552B438061268BE8FBC
:1033BF005222E552B43306126A1E8F5222E552B4DE
:0C33CF004406126CAF8F5222E4F552222B
:10661B007D077F05124E3A500D30000A90052AE097
:10662B00F52BA3E0F52C7D067F02124E3A500C9011
:0E663B00052CE0F529A3E0F52AD21E7F0522EA
:1038DF00302314200F11C21B7D047F01124E3A506A
:1038EF00037F0B227F0A22302414201111D21B7D5B
:1038FF00047F02124E3A50037F0B227F0A227F0869
:10390F001262C950061243B67F0022202308300FDF
:10391F0005C20F7F0522202408301105C2117F0533
:10392F00227D057F06124E3A501EE5394538701834
:10393F009000B5E0FF7C0D7D80125BCA90052EE0F4
:10394F00F538A3E0F53980687D067F06124E3A50B0
:10395F001EE53C453B70189000B6E0FF7C0D7DA046
:10396F00125BCA900530E0F53BA3E0F53C80417D4A
:10397F00077F05124E3A500B300008E52C452B708F
:10398F0002C2007D067F02124E3A5019301E16E514
:10399F002A45297010C21E9000BCE0FF7C0E7D608E
:1039AF00125BCA800B7885E6B405057F0412515966
:0F39BF00E551700875510AD22A1268047F05225B
:1069FC0090053BE0F54E202306201B037F0522204B
:106A0C002406301B037F0522E54ED3940050E77F0C
:026A1C000A224C
:10446B007D077F05124E3A50127D077F05124E3A9B
:10447B004003024510200003024510201B43D22F9E
:10448B007F03122F1A7F0F126E5390000FE0B402AE
:10449B00047F05800990000FE0B403057F01120033
:1044AB00161255C87D027F07124E3A50057F041233
:1044BB006E9A9000A0E0FF7C0A7DE0125BCA7F0F32
:1044CB0022301B4190000FE0FF64026005EF640394
:1044DB0070337F0F126E537F051262C9400BD22FC0
:1044EB007F01122F1A7F028009D22F7F03122F1AFE
:1044FB007F0A1200167D027F07124E3A500A7F0484
:0E450B00126E9A80031255C81255F47F0F22CB
:106D6400201B063023037F1122301B053024027FB1
:026D74001222E9
:1058FB00302352E5484547700C7D087F01124E3A24
:10590B0050037F3722300329E53A70257FA0126EB2
:10591B005390000FE0B401047F01800990000FE069
:10592B00B402057F05120016E4F542C21DC20380C6
:10593B00113025037F14227885E6B405057F031209
:08594B0051597F11227F142243
:1051D300301B1030230D200F0A7F0A126E53C21B9F
:1051E3007F0A22301B4C302449201146300303121E
:1051F3006C1AE54A4549700C7D087F02124E3A50FD
:10520300037F3822300417E53A70137FA0126E53E0
:105213007F02120016E4F542C21DC204801130273A
:10522300037F14227885E6B405057F031251597F65
:105233001222201B1230240F20110CD21BC22F7FED
:0A52430002122F1A7F0A227F1422A4
:10102D0090053DE0F54B7F0F126E53E542B403037F
:10103D007F1422126C1AE4F5427D027F07124E3A9C
:10104D005009E54B70057F04126E87D22A12680491
:10105D00301B0302115EE545700302115E9000A185
:10106D00E0FF7C0B7D00125BCA7C017D001212E754
:10107D0050037F3E227C017D501212B750037F3CFE
:10108D00227C017D581212B750037F3C227C017DDA
:10109D00101212BF50081212CF50037F33227C0161
:1010AD007D201212BF50030211D17C017D28121236
:1010BD00D7500C9000BAE0FF7C0E7D200211DA7C37
:1010CD00017D301212D7500C9000B9E0FF7C0E7DDF
:1010DD00000211DA7C017D40D228E4FF1247C7508F
:1010ED000C7D067F04124E3A50037F4C227C017D0D
:1010FD00381212E750037F44227C017D18C228E488
:10110D00FF1247C7500C7D057F01124E3A50037FE9
:10111D004122E4F55A1255C0EF7803C333CE33CED6
:10112D00D8F91255D3E4FF1247C7501D1255C012FE
:10113D0055E0C0071255C0EF7805C333CE33CED876
:10114D00F91255FFD007125B7F12560A40C77F195F
:10115D0022201B0302125DE546700302125D900012
:10116D00A3E0FF7C0B7D40125BCA7D017F03124E15
:10117D003A40030212157C017D08C2287F011247F7
:10118D00C7500F7F50120016D22F7F02122F1A7FD9
:10119D003F227C017D501212C750037F3D227C01FE
:1011AD007D581212C750037F3D227C017D10121213
:1011BD00DF50081212CF50037F33227C017D2012A5
:1011CD0012DF50129000BBE0FF7C0E7D40125BCA17
:1011DD001267B87F00227C017D40D2287F01124723
:1011ED00C7500C7D067F04124E3A50037F4D227C72
:1011FD00017D18C2287F011247C7500C7D057F0263
:10120D00124E3A50037F43227D027F03124E3A5015
:10121D003CE4F55A1255C0EF7803C333CE33CED824
:10122D00F91255D37F011247C7501D1255C01255E3
:10123D00E0C0071255C0EF7805C333CE33CED8F9D1
:10124D001255FFD007125B7F12560A40C77F192235
:10125D001212EF50081212EF504130003E7885E621
:10126D0070047F0180087885E6B404077F0212516F
:10127D005980257D037F06124E3A501CE557455681
:10128D0070169000AFE0FF7C0C7DC0125BCA90051C
:10129D0032E0F556A3E0F5577F19227D077F051241
:0912AD004E3A50052000027F05B5
:1012B60022D228E4FF1247C722D228E4FF1247C7EA
:1012C60022D2287F011247C7227D077F05124E3A98
:1012D60022D228E4FF1247C722D2287F011247C72D
:1012E60022C228E4FF1247C7227D077F05124E3A25
:0112F60022D5
:1065BE00C218C22F7F02122F1A3025051267B8801B
:1065CE00063027031267DE7D077F05124E3A50060E
:0F65DE002000037F0522900538E0F54E7F1E2236
:10655F00E54E70037F23227D027F07124E3A5009CA
:10656F00E54B70057F04126E87302306200F037FE3
:10657F000A22302408201105D21B7F0A227F1E22F7
:105E9800201B051255C880031255F47D067F011298
:105EA8004E3A5024E5427020201B0B9000ACE0FFD6
:105EB8007C0C7D60800C301B0C9000ADE0FF7C0CEE
:105EC8007D80125BCA7F2822900539E0F54E7F2D30
:015ED80022A7
:0E6E6F007FA0126E53900539E0F54E7F2D2264
:10613D00D22A1268047D027F07124E3A5009E54BB0
:10614D0070057F04126E87E54E601D302306200F0B
:10615D00037F0A2290000FE06401600930240620BD
:0B616D0011037F05227F2D227F3222CC
:10622300301D037F32227D047F06124E3A501FE554
:1062330055455470199000B0E0FF7C0C7DE0125B73
:10624300CA900534E0F554A3E0F5557F3222C22FFE
:086253007F01122F1A7F0022C7
:106D760020210CD221E4FF12055BC2217F00227F75
:026D86003C22AD
:1068990020211FC22F7F02122F1AD2217F401200FE
:1068A90016D201121E0BC2017F40126E53C2217F04
:0568B90019227F3E22C0
:106D990020210BD221D202121C0A1255ED227F3F6B
:016DA90022C7
:106BFF00202115125614122F1A7F40126E537F0147
:0B6C0F0012055BC2217F00227F3D22A6
:106AA20020211912561B122F1A7F10126E53D20177
:0F6AB200E4FF123602C201C2217F19227F412266
:1069940020211D125614122F1A7F40126E53D22F2B
:1069A4007F02122F1AD2027F011236021255ED22F3
:0369B4007F4322FC
:106C340020211412561B122F1AD201E4FF12608B6A
:0A6C4400C201C2217F19227F412204
:1069B70020211D125614122F1A7F40126E53D22F08
:1069C7007F02122F1AD2027F0112608B1255ED221D
:0369D7007F4322D9
:106CAF0020211112561B122F1AD202E4FF12548CFC
:076CBF001255ED227F442273
:10584A00D20F7D027F07124E3A50057F04126E87EF
:10585A0090000FE0FF64016004EFB4030E7F0112B1
:10586A006E537F401258937F01801390000FE0B46B
:10587A00020F7F05126E537F501258937F03126EE8
:10588A00877F50126E537F3922120016C22F126977
:09589A002BE4FD7F07124EC2222F
:1057F0003023037F3922E47885F6C20F90000FE052
:10580000FF64016004EFB4030E7F01126E9A7F40C3
:1058100012583A7F01801890000FE0B402147F0301
:10582000126E9A7F05126E537F5012583A7F031200
:105830006E877F50126E537F0022120016C22F1205
:0A584000692BE4FD7F08124EC2221E
:1068BE00D2117F0A126E537F40120016D22F126928
:1068CE002BE4FD7F07124EC27F03126E877F50129C
:0568DE006E537F002253
:106A1E0030000B9000B8E0FF7C0D7DE0800C200074
:106A2E000E9000B7E0FF7C0D7DC0125BCAB2007FF6
:026A3E0019221B
:10608B008F5AE55A24FF922F12692BE55A70127F13
:10609B0040120016D201E4FD7F09124EC2C20180EC
:1060AB0015E55AB401107F10120016D202E4FD7FE1
:0C60BB0009124EC2C2027F50126E532226
:104F4A00C201C202D20C7F50126E537F8012001629
:104F5A0075420390000FE0B401163023647F0112FA
:104F6A000016302307E542D3940050F67F01804EA5
:104F7A0090000FE0FF64026005EF64037043302382
:104F8A00267F02126E53D22F7F03122F1A7F051229
:104F9A000016302307E542D3940050F6C22F7F0251
:104FAA00122F1A7F0580173024177F02120016303D
:104FBA00240AE542D3940040033023F37F02126EA1
:084FCA0053E542708EC20C2277
:03000000026B9000
:106B9000758E0078FEE4F6D8FD9000007FFF7E1F22
:0D6BA000E4F0A3DFFCDEFA758188024C03EF
:103ABC00C2D530F707B2D563F0FF05F030E70CB292
:103ACC00D5F4048463F0FF05F080018430D502F452
:023ADC000422C2
:103ADE00EF8DF0A4A8F0CF8CF0A428CE8DF0A42EFC
:023AEE00FE22B6
:103AF000BC000BBE0029EF8DF084FFADF022E4CCBA
:103B0000F875F008EF2FFFEE33FEEC33FCEE9DEC82
:103B1000984005FCEE9DFE0FD5F0E9E4CEFD22EDC8
:103B2000F8F5F0EE8420D21CFEADF075F008EF2F12
:103B3000FFED33FD4007985006D5F0F222C398FD03
:053B40000FD5F0EA22A0
:103B4500EB9FF5F0EA9E42F0E99D42F0E89C45F0D6
:013B5500224D
:103B56007401FF3395E0FEFDFC080808E6CF2FF65A
:103B660018E6CE3EF618E6CD3DF618E6CC3CF62233
:0C3B7600A42582F582E5F03583F583225A
:103B8200D083D082F8E4937012740193700DA3A3D2
:103B920093F8740193F5828883E4737402936860E6
:063BA200EFA3A3A380DFE6
:106DAA00EFC39461400AEF947B5005EF24E0FF2281
:016DBA0022B6
:00000001FF
